:020000040800F2
:1000000000070020F102000811340008C93300087D
:10001000F1330008C9330008E9330008F30200088F
:10002000F3020008F3020008F302000899440008F4
:10003000F3020008F3020008F3020008F3020008CC
:10004000F3020008F3020008F3020008F3020008BC
:10005000F3020008F30200084D6500087965000806
:10006000A5650008D1650008FD6500085D4500082C
:1000700085450008B1450008DD450008094600082F
:10008000314600085D460008F30200087933000895
:10009000A13300088D330008B53300082966000835
:1000A000F3020008F3020008F3020008F30200085C
:1000B000F3020008F3020008F3020008F30200084C
:1000C000F3020008F3020008F3020008F30200083C
:1000D000F302000801670008F3020008F3020008B9
:1000E0008D660008F3020008F3020008F30200081E
:1000F000F3020008F3020008F30200088946000832
:10010000F3020008F302000829670008F302000860
:10011000F3020008F3020008F3020008F3020008EB
:10012000B5460008DD4600080947000835470008C5
:1001300061470008F3020008F3020008F302000818
:10014000F3020008F3020008F3020008F3020008BB
:1001500089470008B5470008E1470008F302000896
:10016000F3020008F3020008F3020008F30200089B
:10017000F3020008F3020008F3020008F30200088B
:10018000F3020008F3020008F302000815670008F4
:10019000F3020008F3020008F3020008F30200086B
:1001A000F3020008F3020008F3020008F30200085B
:1001B000F3020008F3020008F3020008F30200084B
:1001C000F3020008F3020008F3020008F30200083B
:1001D000F3020008F3020008F3020008F30200082B
:1001E000F3020008F3020008F3020008F30200081B
:1001F000F3020008F3020008F3020008F30200080B
:10020000F3020008F3020008F3020008F3020008FA
:10021000F3020008F3020008F3020008F3020008EA
:10022000F3020008F3020008F3020008F3020008DA
:10023000F3020008F3020008F3020008F3020008CA
:10024000F3020008F3020008F3020008F3020008BA
:10025000F3020008F3020008F3020008F3020008AA
:10026000F3020008F3020008F3020008F30200089A
:10027000F3020008F3020008F3020008F30200088A
:10028000F3020008F3020008F3020008F30200087A
:10029000F3020008F3020008F3020008F30200086A
:1002A000F3020008F3020008F3020008F30200085A
:1002B000F3020008F3020008F3020008F30200084A
:1002C000F3020008F3020008F3020008F30200083A
:1002D000F3020008F3020008F3020008F30200082A
:1002E000CD16000800000000000000000000000023
:1002F00002E000F000F8FEE772B6374880F30888A5
:10030000364880F3098836483649086040F20000D4
:10031000CCF200004EF63471CEF200010860BFF35B
:100320004F8FBFF36F8F40F20000C0F2F0004EF627
:100330008851CEF200010860BFF34F8FBFF36F8F7B
:100340004FF00000E1EE100A4EF63C71CEF20001D3
:100350000860062080F31488BFF36F8F05F086FCD9
:1003600005F0C2FE4FF055301F491B4A91423CBF79
:1003700041F8040BFAE71D49184A91423CBF41F885
:10038000040BFAE71A491B4A1B4B9A423EBF51F82D
:10039000040B42F8040BF8E700201849184A914270
:1003A0003CBF41F8040BFAE705F09EFC05F022FF84
:1003B000144C154DAC4203DA54F8041B8847F9E796
:1003C00000F042F8114C124DAC4203DA54F8041B11
:1003D0008847F9E705F086BC0007002000230020CD
:1003E0000000000808ED00E00001002000070020E8
:1003F000486C0008002300203C23002040230020FC
:1004000004710020E0020008E4020008E402000891
:10041000E40200082DE9F04F2DED108AC1F80CD050
:10042000D0F80CD0BDEC108ABDE8F08F002383F328
:1004300011882846A047002004F072FFFEE704F070
:10044000F7FE00DFFEE70000F8B501F055F901F016
:1004500003FA01F04DFB05F065FB074605F0FCFBD8
:100460000546A8BB1F4B9F4232D001339F4232D07A
:1004700027F0FF021C4B9A4230D12E4642F21074F4
:10048000F8B200F06FFF00F073FF08B100242646B9
:1004900001F0BEFD20B10024032000F079F82646CB
:1004A00035B1124B9F4203D0002405F0CDFB264608
:1004B000002005F041FB0EB100F080F801F0EAFAEF
:1004C00000F08AFF204600F00BF900F077F8F9E71A
:1004D0002E460024D7E704460126D4E7064641F21B
:1004E0008834D0E7010007B0000008B0263A09B010
:1004F00008B501F07DF9A0F120035842584108BD2C
:1005000007B541F21203022101A8ADF8043001F051
:100510008DF903B05DF804FB38B5302383F31188FF
:10052000174803680BB104F0B9FF0023154A4FF4D4
:100530007A71134804F0A8FF002383F31188124C4A
:10054000236813B12368013B2360636813B16368B8
:10055000013B63600D4D2B7833B963687BB9022092
:1005600001F02EFA322363602B78032B07D16368E6
:100570002BB9022001F024FA4FF47A73636038BD7E
:100580004023002019050008602400205823002083
:10059000084B187003280CD8DFE800F008050208A3
:1005A000022001F00BBA022001F006BA024B002231
:1005B0005A6070475823002060240020F8B501F0ED
:1005C00027FD30B13E4B03221A7000223D4B5A608A
:1005D000F8BD3D4B3D4A1C4619680131F8D0043343
:1005E0009342F9D162683A4B9A42F1D9394B9B68F0
:1005F00003F1006303F580239A42E9D205F0F8FA8B
:1006000005F00AFB002001F04DF90220FFF7C0FFC2
:10061000314B00219A6C99641A6F19671A6FDA6C62
:10062000D9645A6F59675A6F1A6D19659A6F99672D
:100630009B6F72B64FF0E023C3F8084DD4E9000475
:10064000BFF34F8FBFF36F8F244AC2F88410BFF3FC
:100650004F8F536923F480335361BFF34F8FD2F828
:10066000803043F6E076C3F3C905C3F34E335B0134
:1006700003EA060C29464CEA81770139C2F8747204
:10068000F9D2203B13F1200FF2D1BFF34F8FBFF30C
:100690006F8FBFF34F8FBFF36F8F536923F4003316
:1006A00053610023C2F85032BFF34F8FBFF36F8FF7
:1006B000302383F31188854680F30888204787E735
:1006C00058230020602400200000040820000408B3
:1006D000FFFF0308002300200045025800ED00E062
:1006E0002DE9F04F93B0B74B2022FF2100900AA8CC
:1006F0009D6801F079F9B44A1378A3B90121B34890
:1007000011700360302383F3118803680BB104F088
:10071000C5FE0023AE4A4FF47A71AC4804F0B4FE33
:10072000002383F31188009B13B1AA4B009A1A602F
:10073000A94A1378032B03D000231370A54A5360F2
:100740004FF0000A009CD3465646D146012001F0E6
:1007500035F924B19F4B1B68002B00F02C82002040
:1007600001F046F80390039B002B01DA00F088FEAD
:10077000039B002BEDDB012001F01EF9039B213BC5
:100780001F2BE3D801A252F823F000BF0D08000888
:1007900035080008C90800084D0700084D07000883
:1007A0004D0700085B0900082B0B0008450A0008EC
:1007B000A70A0008CF0A0008F50A00084D0700083C
:1007C000070B00084D070008790B0008AD0800086A
:1007D0004D070008BD0B000819080008AD08000807
:1007E0004D070008A70A00084D0700084D0700083C
:1007F0004D0700084D0700084D0700084D07000889
:100800004D0700084D070008C90800080220FFF73F
:100810006FFE002840F0F981009B022105A8BAF183
:10082000000F08BF1C4641F21233ADF8143000F03F
:10083000FDFF8BE74FF47A7000F0DAFF071EEBDB69
:100840000220FFF755FE0028E6D0013F052F00F2F9
:10085000DE81DFE807F0030A0D10133605230421BB
:1008600005A8059300F0E2FF17E004215548F9E7D9
:1008700004215A48F6E704215948F3E74FF01C08D1
:10088000404608F1040801F00FF80421059005A87E
:1008900000F0CCFFB8F12C0FF2D101204FF000098D
:1008A00000FA07F747EA0B0B5FFA8BFB01F0E8F859
:1008B00026B10BF00B030B2B08BF0024FFF720FE23
:1008C00044E704214748CDE7002EA5D00BF00B03E9
:1008D0000B2BA1D10220FFF70BFE074600289BD06F
:1008E0000120002600F0DEFF0220FFF751FE1FFA74
:1008F00086F8404600F0E6FF0446B0B10399404652
:100900000136A1F140025142514100F0F3FF0028AD
:10091000EDD1BA46044641F21213022105A83E4623
:10092000ADF8143000F082FF10E725460120FFF7F4
:100930002FFE244B9B68AB4207D9284600F0B4FF3A
:10094000013040F067810435F3E70025224BBA46B9
:100950003E461D701F4B5D60A8E7002E3FF45CAF64
:100960000BF00B030B2B7FF457AF0220FFF710FEA9
:10097000322000F03DFFB0F10008FFF64DAF18F057
:1009800003077FF449AF0F4A08EB050392689342CF
:100990003FF642AFB8F5807F3FF73EAF124BB84508
:1009A000019323DD4FF47A7000F022FF0390039A45
:1009B000002AFFF631AF039A0137019B03F8012BA0
:1009C000EDE700BF002300205C240020402300202E
:1009D000190500086024002058230020042300206B
:1009E000082300200C2300205C230020C820FFF7F0
:1009F0007FFD074600283FF40FAF1F2D11D8C5F12A
:100A000020020AAB25F0030084494245184428BF60
:100A10004246019200F0D6FF019AFF217F4800F084
:100A2000E3FF4FEAA803C8F387027C4928460193F5
:100A300000F0E2FF064600283FF46DAF019B05EB96
:100A4000830533E70220FFF753FD00283FF4E4AEAF
:100A500000F062FF00283FF4DFAE0027B846704B7D
:100A60009B68BB4218D91F2F11D80A9B01330ED0A7
:100A700027F0030312AA134453F8203C0593404681
:100A8000042205A9043701F0ADFA8046E7E73846AD
:100A900000F00AFF0590F2E7CDF81480042105A8C4
:100AA00000F0C4FE02E70023642104A8049300F0D0
:100AB000B3FE00287FF4B0AE0220FFF719FD002836
:100AC0003FF4AAAE049800F01DFF0590E6E700236E
:100AD000642104A8049300F09FFE00287FF49CAEDC
:100AE0000220FFF705FD00283FF496AE049800F0C1
:100AF0000BFFEAE70220FFF7FBFC00283FF48CAE77
:100B000000F01AFFE1E70220FFF7F2FC00283FF4B3
:100B100083AE05A9142000F015FF074604210490B8
:100B200004A800F083FE3946B9E7322000F060FEE9
:100B3000071EFFF671AEBB077FF46EAE384A07EBB7
:100B40000903926893423FF667AE0220FFF7D0FC9C
:100B500000283FF461AE27F003074F44B9453FF446
:100B6000A5AE484609F1040900F09EFE0421059057
:100B700005A800F05BFEF1E74FF47A70FFF7B8FCD0
:100B800000283FF449AE00F0C7FE002844D00A9B7D
:100B900001330BD008220AA9002000F02DFF002805
:100BA0003AD02022FF210AA800F01EFFFFF7A8FC80
:100BB0001C4804F0BBFB13B0BDE8F08F002E3FF4DF
:100BC0002BAE0BF00B030B2B7FF426AE002364211E
:100BD00005A8059300F020FE074600287FF41CAE10
:100BE0000220FFF785FC804600283FF415AEFFF792
:100BF00087FC41F2883004F099FB059800F05EFF15
:100C000046463C4600F03CFFA0E506464EE64FF067
:100C1000000901E6BA467EE637467CE65C23002002
:100C200000230020A0860100094A49F269001368E8
:100C300099B21B0C00FB013344F250611360054B69
:100C4000186882B2000C01FB0200186080B2704785
:100C500014230020102300200021102210B5044688
:100C600000F0C2FE034B03CB206061601868A060F7
:100C700010BD00BF00E8F11FF0B5ADF54F7D4FF49A
:100C8000C47207460D466CAC0021204600F0ACFE55
:100C900002F0C6FB4FF47A72254BB0FBF2F01860FD
:100CA00093E80700022384E807000DF5E97023822A
:100CB000FFF7D2FF41F204331E4907A8238405F051
:100CC000BFFD15230DF2E3220DF12C0C84F8323117
:100CD00007AB1E46083203CE664542F8080C42F8C0
:100CE000041C3346F5D130681060204633790DAED0
:100CF00013713146012200F05BFF002380B2E97ED0
:100D00000393AB7E029305F1190301930123009332
:100D100005A3D3E90023CDE90460384602F08CFF37
:100D20000DF54F7DF0BD00BF9E6AC421818A46EE5D
:100D300068240020506800082DE9F0412C4CDAB0FE
:100D400080460D46237A5BBB27A9284601F054F85C
:100D50000746002842D19DF89D60C82E3ED8014626
:100D60004FF4A662204600F03FFE4FF480733246F7
:100D70000DF19E01C4F8F8314FF4007304F109003D
:100D80002644C4F80C334FF44073C4F8203400F008
:100D900019FE9DF89C30777223720BB9EB7E23729B
:100DA00006AC8122002127A800F01EFE0122214668
:100DB00027A801F067F8002380B2E97E0393AB7E99
:100DC000029305F1190301932823CDE90440009310
:100DD000404605A3D3E9002302F02EFF5AB0BDE838
:100DE000F08100BFAFF3008026417272DF25D7B7D4
:100DF000B0340020F0B5254E4FF48A75F1B00024D0
:100E000005FB006596F8D830D822214685F8DC30FD
:100E10003AA885F8E84006AF00F0E6FD06F10900C3
:100E200000F0DAFDD5F8E430C2B206F109018DF820
:100E3000F0000DF1F100CDE93A3400F0C3FD394680
:100E400001223AA801F054F8082380B2317ACDE9A2
:100E5000047001270E48CDE9023706F1D80301934B
:100E60003023009307A3D3E9002302F0E5FEA0425C
:100E700006DD02F0D5FAC5F8E000384671B0F0BDE5
:100E80002046FBE778F6339F93CACD8DB03400201F
:100E9000803400202DE9F04F274F87B0DFF8A48081
:100EA000264E384602F0F4FE034600283CD00024CB
:100EB000234DADF81440A1460294A246CDE9034467
:100EC000027B8DF8142003AA9968406803C21B684E
:100ED00043F0004302932B6804F23454D3F810B06B
:100EE00002F0A0FA10EB0802CDF800A0284605F5A4
:100EF000A65541F1000302A9D84740F6682300280F
:100F0000C8BF49F0010910359C42E4D1B9F1000F86
:100F100005D0384602F0C0FE86F800A0C1E733785D
:100F2000072B04D80133337007B0BDE8F08F0248B7
:100F300002F0B2FEF8E700BF80340020E53900205F
:100F4000E839002040420F0070B50D4614461E4699
:100F500002F0CEFD50B9022E10D1012C0ED112A3F9
:100F6000D3E900230120C5E9002307E0282C10D095
:100F700005D8012C09D0052C0FD0002070BD302CD5
:100F8000FBD10BA3D3E90023ECE70BA3D3E90023A8
:100F9000E8E70BA3D3E90023E4E70BA3D3E900239D
:100FA000E0E700BFAFF30080401DA12026812A0B9F
:100FB00078F6339F93CACD8D9E6AC421818A46EE0E
:100FC00026417272DF25D7B7F017304A39059E5691
:100FD00038B505460E4C0021013500F08BFCA4F815
:100FE0002C55B4F82C0500F06DFC78B1B4F82C0544
:100FF00000F078FC014648B9B4F82C0500F07AFC02
:10100000B4F82C350133A4F82C35EAE738BD00BF1D
:10101000B0340020F8B50E4C02260E4FA4F58053D4
:1010200043F8407C237E3BB965692DB1284601F029
:101030006DF8284601F0A6F92046A4F5A65401F063
:1010400065F8012EA4F1100400D1F8BD0126E5E7F2
:10105000F85E0020086900082DE9F04F8FB00546C2
:101060000C4600AF02F044FD00284BD1237E022B3A
:101070001BD1E38A012B18D102F0D2F90646FFF703
:10108000D3FD03464FF4C87006F51676DFF8D0821C
:10109000B3FBF0F202FB103316FA83F3C8F800300A
:1010A000E37E33B9A74B00221A703C37BD46BDE83A
:1010B000F08F07F12401204600F052FE0028F4D101
:1010C00007F11400FFF7C8FD97F8264007F1140157
:1010D00007F12700224605F081FB0028E2D10F2C02
:1010E00008D8984B1C70D8F80030A3F51673C8F8D0
:1010F0000030DAE797F824100029D6D0284602F00D
:10110000EFFCD2E7E38A282B33D010D8012B2BD069
:10111000052BCAD1BFF34F8F8B498C4BCA6802F4A1
:10112000E0621343CB60BFF34F8F00BFFDE7302B6E
:10113000BBD1874EE17E327A9142B6D1607E314694
:10114000002291F8DC50854200F0AD80013201F5BB
:101150008A71042AF5D1326840F6B831FA328A42EF
:1011600094BF32603160A0E721462846FFF784FD36
:101170009BE721462846FFF7DFFD96E7B2F8EC50E3
:101180007B6005F103094FEA99094FEA8902D11DF5
:10119000C908A8EBC10300219D46EB46584600F064
:1011A00023FC04F1EE012A465846314400F00AFCC3
:1011B0007B6813B9012000F075FB96F8D20000F0AF
:1011C00081FB044630B9307200F0A6FB204600F0E7
:1011D00069FBB0E0D6F8D4203AB996F8D200B6F858
:1011E0002C25824201D8FFF7F3FED6F8D4202A44FA
:1011F000944208D296F8D200B6F82C2501308242EB
:1012000001D8FFF7E5FE5FFA89F25946706800F0F1
:10121000F3FB08B9C54679E0726896F8D2002A4413
:101220007260D6F8D42005EB0209C6F8D49000F01D
:1012300049FB814509D396F8D220D6F8D400013273
:10124000001B86F8D220C6F8D400FF2D0FD800244A
:10125000347200F061FB204600F024FB00F0D8FE61
:101260003C4B188108B9FFF7A9F9C5461DE7BB68D3
:1012700096F8D9000AFB0362FB68D2F8E41082F802
:10128000E83001F58061C2F8E030C2F8E410FFF701
:10129000B1FDFFF7FFFD96F8D920013202F00302FD
:1012A00086F8D920B6E74FF48A7A20460AFB02F581
:1012B00005F1EA01314400F04FFEF86000287FF4A8
:1012C000F4AE0122354485F8E82002F0A9F8D5F8FB
:1012D000E020D6ED007A801A40F6B832B8EE677A90
:1012E000DFED1D6A192838BF1920904228BF10462B
:1012F00007EE900AF8EEE77A67EEA67ADFED176A56
:10130000E7EE267AFCEEE77AC6ED007A96F8D93059
:1013100071680AFB03F4BB60321992F8E8505DB1C2
:10132000D2F8E430E8468B423FF428AF002182F83F
:10133000E810C2F8E010C5467368064A9B0A0133FC
:101340001381B2E67934002000ED00E00400FA05D4
:10135000B034002068240020CDCCCC3D6666663FCA
:101360007C340020014B1870704700BF74240020AB
:1013700038B54FF00054144B22689A4222D1607D58
:10138000F8B1124B0025C922114918701148237D6C
:101390000930C0F8DB5000F8013C4FF48073C0F80E
:1013A000EF314FF40073C0F803334FF44073C0F8CB
:1013B000173400F007FBE0222946204600F014FB1A
:1013C000012038BD0020FCE79AAD44C574240020FC
:1013D00016000020B034002037B500F019FE1F4C75
:1013E0001F4D022301221F496B712368288120466B
:1013F00004F580545B6898470122D4F8D03404F592
:101400009A6018495B689847002317494FF4805247
:101410000193164B16480093164B02F039FB164BFE
:10142000197811B1124802F05BFB01F0F9FF044694
:10143000FFF7FAFB4FF4C873B0FBF3F202FB1303A0
:1014400004F5167010FA83F00C4B186004F004FCDD
:1014500008B10F232B8103B030BD00BFE839002055
:101460006824002040420F0078240020490F000823
:101470008034002059100008742400207C3400209F
:101480002DE9F04F00252DED028B93B00DF12C08C6
:101490004FF0010ADFF814B2FFF7FCFC0A95ADF833
:1014A00034500B95C8F804509FED798B00267E4C84
:1014B000374623680DF11D0207A920468DF81CA0B0
:1014C0008DF81D508DED008BD3F808900023C84790
:1014D0009DF81C90B9F1000F1ED0102200210EA81B
:1014E00000F082FA236808AA0AA95F6920460DF174
:1014F0001E03B8470FAB4F4698E8030083E803008C
:101500009DF834300EA958468DF844300A9B0E934E
:10151000DDE9082302F09EFD06F2345640F668230A
:1015200004F5A6549E4204F11004C2D1002FBDD18F
:101530005E4802F0DDFA00283FD15D4E01F070FFF9
:101540003368984239D301F06BFF0446FFF76CFB18
:101550004FF4C8738DF82870B0FBF3F202FB13034D
:1015600004F5167010FA83F03060524E377817B9D0
:1015700001238DF82830C7F110040EA8FFF76CFB8B
:101580000EABE4B20DF12900D919062C28BF0624B0
:101590002246013400F016FA0AABE4B24348039342
:1015A000182304940293444B0193012300933AA31C
:1015B000D3E9002302F0E2FA357001F031FF3F4A2F
:1015C0003F4C1368C31AB3F57A7F2FD3106001F034
:1015D00029FF02460B46354802F068FB334802F00B
:1015E00087FA18B3237A0EAF364E002B14BF0323AD
:1015F0000223737101F014FF4FF47A73012239460C
:10160000B0FBF3F03060304600F082FB182380B26C
:1016100002932D4B019340F25513CDE903700093D3
:1016200022481FA3D3E9002302F0A8FA237A93B13A
:1016300001F0F6FE002607464FF48A7894F8D900A8
:10164000304400F0030008FB004393F8E82072B137
:101650000136042EF2D1C82003F068FE237A002B55
:101660007FF414AF13B0BDEC028BBDE8F08FD3F85C
:10167000E02042B12368BA1AFA2B38BFFA230533A7
:10168000B2EB430FE4D3FFF7B5FB0028E0D1E2E76C
:101690000000000000000000401DA12026812A0B50
:1016A000F1C6A7C1D068080FE839002080340020B7
:1016B0007C3400207934002078340020E039002088
:1016C000B034002068240020E439002008B5064822
:1016D00001F066F9054801F063F9054A0549002063
:1016E000BDE8084005F066B8E8390020B84E002093
:1016F000E063002015100008F8B50A25204C0122EF
:101700004FF400712046192703F056F920460122B4
:101710004FF4807103F050F94FF480766520013862
:1017200025D00822A2F10801B646332905D84FF08A
:10173000000C66834FF000730DE0A1F13403668363
:10174000B3FBF7FC07FB1C33002B0CBF4FF0010C65
:101750004FF0000CEED1013143EA4C238A42A361E1
:10176000A4F818E0E1D10832A02AD8D0DAE7013D88
:1017700042F2107003F0DAFD15F0FF05BFD1F8BD9D
:10178000000402582DE9F84F4FF47A7306460D46CF
:10179000002402FB03F7DFF85080DFF8509098F93F
:1017A00000305FFA84FA5A1C01D0A34212D159F8D2
:1017B00024002A4631460368D3F820B03B46D84778
:1017C000854207D1074B012083F800A0BDE8F88FC0
:1017D0000124E4E7002CFBD04FF4FA7003F0A6FDDF
:1017E0000020F3E7CC630020182300201C230020F6
:1017F000002307B5024601210DF107008DF80730DF
:10180000FFF7C0FF20B19DF8070003B05DF804FBAF
:101810004FF0FF30F9E700000A46042108B5FFF752
:10182000B1FF80F00100C0B2404208BD074B0A463C
:1018300030B41978064B53F82140014623682046FE
:10184000DD69044BAC4630BC604700BFCC63002070
:101850001C230020A086010070B5104C0025104EFE
:1018600003F034FF20803068238883420CD80025A1
:101870002088013803F026FF23880544013BB5F595
:10188000802F2380F4D370BD03F01CFF3368054420
:101890000133B5F5802F3360E5D3E8E7CE63002050
:1018A0008863002003F0E0BF00F1006000F58020B5
:1018B0000068704700F10060920000F5802003F09E
:1018C00061BF0000054B1A68054B1B889B1A8342B9
:1018D00002D9104403F0F6BE002070478863002050
:1018E000CE630020024B1B68184403F0F1BE00BF1A
:1018F00088630020024B1B68184403F0FBBE00BF46
:10190000886300200020704700F1FF5000F58F1021
:10191000D0F8000870470000064991F8243033B130
:1019200000230822086A81F82430FFF7C3BF012092
:10193000704700BF8C630020014B1868704700BFE0
:101940000010005C194B01380322084470B51D6873
:10195000174BC5F30B042D0C1E88A6420BD15C68F7
:101960000A46013C824213460FD214F9016F4EB170
:1019700002F8016BF6E7013A03F10803ECD181426A
:101980000B4602D22C2203F8012B0424094A1688A4
:10199000AE4204D1984284BF967803F8016B013CB3
:1019A00002F10402F3D1581A70BD00BF0010005CB0
:1019B000242300209468000870470000704700004E
:1019C00070470000002310B5934203D0CC5CC45490
:1019D0000133F9E710BD000003460246D01A12F9A0
:1019E000011B0029FAD1704702440346934202D0FA
:1019F00003F8011BFAE770472DE9F8431F4D144621
:101A00000746884695F8242052BBDFF870909CB3B7
:101A100095F824302BB92022FF2148462F62FFF78A
:101A2000E3FF95F824004146C0F1080205EB800071
:101A3000A24228BF2246D6B29200FFF7C3FF95F814
:101A40002430A41B17441E449044E4B2F6B2082E7E
:101A500085F82460DBD1FFF75FFF0028D7D108E0CD
:101A60002B6A03EB82038342CFD0FFF755FF002898
:101A7000CBD10020BDE8F8830120FBE78C63002078
:101A8000024B1A78024B1A70704700BFCC630020DB
:101A90001823002010B5074C4FF4E13306492068A5
:101AA0000B6003F00BFB60680349BDE8104003F0D6
:101AB00005BB00BF1C230020B4630020094B182283
:101AC000002110B504461846FFF78EFF064A074B63
:101AD00001461278046053F82200BDE8104003F07C
:101AE000EDBA00BFB4630020CC6300201C230020AB
:101AF000F8B571B6002301201A46194602F00EFF10
:101B00000446802003F04EFF002849D00025254AD6
:101B100080274FF4D06C3D26136913F0C06F26D197
:101B2000D2F8103113F0C06F21D1236805F10061A4
:101B300099602368D86023685F602368C3F800C099
:101B400021680B6843F001030B6021680B6823F0E8
:101B50001E030B6021680B68DB07FCD4237B8035F8
:101B6000616806FA03F3B5F5001F0B60D4D1204677
:101B700002F00AFFB5F5001F11D000240A4E0B4DEC
:101B8000012003F071FE3388A34205D92868204460
:101B9000013403F0AFFDF6E7002003F065FE61B607
:101BA000F8BD00BF00200052CE63002088630020F3
:101BB0002DE9F3470D46044600219046284640F2A1
:101BC0007912FFF711FF234620220021284604F155
:101BD000220702F0E1F9231D022220212846C02617
:101BE00002F0DAF9631D03222221284602F0D4F91B
:101BF000A31D03222521284602F0CEF904F1080393
:101C000010222821284602F0C7F904F11003082207
:101C10003821284602F0C0F904F1110308224021BE
:101C2000284602F0B9F904F1120308224821284697
:101C300002F0B2F904F1140320225021284602F0E8
:101C4000ABF904F1180340227021284602F0A4F9F0
:101C500004F120030822B021284602F09DF904F186
:101C600021030822B821284602F096F931460836A9
:101C70003B4608222846013702F08EF9B6F5A07FD0
:101C8000F4D194F83230314604F1330A00268DF84D
:101C9000073008220DF10703284602F07DF99DF870
:101CA00007304FEAC6099E4209F5A47720D394F87D
:101CB0003231502B28BF50238DF80730B8F1000F78
:101CC00008D1394609F24F170DF1070307222846BC
:101CD00002F062F9002604F233149DF8073007EB96
:101CE000C6019E420DD30731C80802B0BDE8F08797
:101CF0000AEB0603082239462846013602F04CF961
:101D0000CDE7A31908222846013602F045F9E4E799
:101D100013B50446084600212022234601900160A5
:101D2000C0F8031002F038F9231D01980222202187
:101D300002F032F9631D01980322222102F02CF9EE
:101D4000A31D01980322252102F026F9019804F130
:101D500008031022282102F01FF9072002B010BD4D
:101D6000F7B5047F05460E462CB1838A122B02D9A3
:101D7000012003B0F0BD0023072228460096194633
:101D800001F0CEFF731C0122072100932846002397
:101D900001F0C6FFD4B9B31C0522082128460093E0
:101DA00023460D2401F0BCFFB378102BE0D8374652
:101DB000BB1BB278934210D307342B7FA88AE40868
:101DC000B3B9844294BF00200120D2E7AB8A082433
:101DD000DB00083BDB08B370E6E7FB1C214608226A
:101DE0002846009300230834013701F099FFDFE70C
:101DF000201A18BF0120BCE7F7B5047F05460E4640
:101E00002CB1838ACA2B02D9012003B0F0BD002374
:101E1000082228460096194601F082FF731CD4B9A7
:101E200008220093234610241146284601F078FF2B
:101E30007378C82BE8D801235F1C7278013B93426A
:101E400010D307342B7FA88AE408B3B9844294BF27
:101E500000200120D9E7AB8A0824DB00083BDB081F
:101E60007370E5E7F3192146082228460093002302
:101E700001F056FF08343B46DEE7201A18BF012068
:101E8000C3E70000F7B50D46044600211646284674
:101E90008122FFF7A9FD234608220021284602F0EF
:101EA0007BF894F901206378002AB8BF7F238DF86E
:101EB00007309EB90F270DF1070307220821284696
:101EC00002F06AF8002602349DF8073007EBC601DD
:101ED0009E4205D30731C80803B0F0BD0827F1E7DB
:101EE000A31908222846013602F056F8ECE7000054
:101EF000F7B50E460546002114463046CE22FFF7C0
:101F000073FD2B4628220021304602F045F82B7A3B
:101F1000C82B28BFC8238DF807308CB930240DF1A9
:101F2000070308222821304602F036F82F467B1B93
:101F30009DF80720934205D3E01DC00803B0F0BD13
:101F40002824F3E707F10903214608223046083424
:101F5000013702F021F8EAE7F7B5047F05460E469F
:101F600034B1838AB3F5827F02D9012003B0F0BD7A
:101F70000123102200212846009601F0D1FEDCB991
:101F8000B31C09221021284600932346192401F08E
:101F9000C7FE7388B3F5807FE7D83746BB1B7288CE
:101FA000934210D307342B7FA88AE408B3B9844244
:101FB00094BF00200120D9E7AB8A1024DB00103B3E
:101FC000DB087380E5E73B1D214608222846009385
:101FD00000230834013701F0A3FEDFE7201A18BF01
:101FE0000120C3E730B50A44084D91420DD011F8E5
:101FF000013B5840082340F30004013B2C4013F000
:10200000FF0384EA5000F6D1EFE730BD2083B8ED3E
:10201000F7B5384A6B46106851686A4603C308230F
:102020003549364804F0EAFB0446002833D10A2536
:10203000334A6B46106851686A4603C30823314926
:102040002E4804F0DBFB0446002849D00369B3F5B1
:10205000E01F45D8B0F8661040F2134291423FD1DC
:10206000294A024402F15C018B4239D35C3B23498B
:1020700000209E1AFFF7B6FF04F1640107463246BE
:102080000020FFF7AFFFA3689F4229D1E368984281
:1020900008BF002524E00369B3F5E01F27D8418B72
:1020A00040F21342914220D1174A024402F110013A
:1020B0008B4218D3103B114900209D1AFFF792FF65
:1020C00004F1180106462A460020FFF78BFFA3689B
:1020D0009E4202D1E368984201D00D25A8E7002571
:1020E000284603B0F0BD1025A2E70C25A0E70B257C
:1020F0009EE700BFA4680008DCFF1B000000040886
:10210000AD68000890FF1B000800FCF710B5037CC9
:10211000044613B9006803F079FC204610BD0000A6
:102120000023BFF35B8FC360BFF35B8FBFF35B8F95
:102130008360BFF35B8F7047BFF35B8F0068BFF3B3
:102140005B8F704770B505460C30FFF7F5FF04460E
:1021500005F108063046FFF7EFFFA04206D96D688B
:102160003046FFF7E9FF2544281A70BD3046FFF7D7
:10217000E3FF201AF9E7000070B505464068A0B1FA
:1021800005F10C0605F10800FFF7D6FF04463046BE
:10219000FFF7D2FF844204F1FF34304694BF6D68EC
:1021A0000025FFF7C9FF2C44201A70BD38B50C4636
:1021B0000546FFF7C7FFA04210D305F10800FFF75F
:1021C000BBFF04446868BFF35B8FB4FBF0F100FB16
:1021D00011440120AC60BFF35B8F38BD0020FCE7E9
:1021E0002DE9F041144607460D46FFF7C5FF84422E
:1021F00028BF0446D4B1B84658F80C6B4046FFF7E8
:102200009BFF3044286040467E68FFF795FF331AF5
:102210009C4203D801206C60BDE8F081A41B6B6078
:102220003B682044AB60E8600220F5E72046F3E716
:1022300038B50C460546FFF79FFFA04210D305F1C5
:102240000C00FFF779FF04446868BFF35B8FB4FBB1
:10225000F0F100FB11440120EC60BFF35B8F38BD4F
:102260000020FCE72DE9FF418846694607466C4699
:10227000FFF7B6FF002506B204EBC606B4420AD04B
:10228000626808EB050120680834FFF79BFB54F8EF
:10229000043C1D44F2E729463846FFF7C9FF2846AB
:1022A00004B0BDE8F0810000F8B505460C300F46DB
:1022B000FFF742FF05F1080604463046FFF73CFFF2
:1022C000A042304688BF6C68FFF736FF201A38609E
:1022D00020B12C683046FFF72FFF2044F8BD0000E6
:1022E00073B5144606460D46FFF72CFF8442019055
:1022F00028BF0446DCB101A93046FFF7D5FF019B9A
:1023000033B93268C5E90233C5E9002401200CE085
:102310009C42286038BF0194019884426860F5D9D6
:102320003368241A0220AB60EC6002B070BD204616
:10233000FBE700002DE9FF410F4669466C46FFF7B9
:10234000CFFF00B2002604EBC005AC4209D0D4F8A0
:102350000480B81954F8081B42464644FFF732FB84
:10236000F3E7304604B0BDE8F081000038B505461B
:10237000FFF7E0FF044601462846FFF717FF204617
:1023800038BD000008B103F041BB70477047000042
:1023900010B41346026814680022A4465DF8044B8A
:1023A0006047000000F5805090F869047047000015
:1023B00000F5805090F862047047000000F58050EE
:1023C00090F96804704700004E207047302383F373
:1023D000118800F58052D2F8AC34D2F8A804184421
:1023E000D2F8A4341844D2F88C341844D2F89C346F
:1023F0001844D2F898341844002383F311887047A6
:1024000000F58050C0F86414012070472DE9FF47A3
:102410000C4600F580510546BDF8308091F8620405
:1024200098B1D1F888040130C1F88804206886008A
:1024300006D4207B08280BD9667B0EB10F2807D95C
:10244000D1F88C340133C1F88C344FF0FF30A9E05F
:10245000302080F31188E86BD0F8C47017F40017AF
:1024600013D0D1F890040130C1F89004D1F894143D
:10247000002940F09A8021462846CDF8008001F0DE
:1024800019F8002383F311888CE0D0F8C4604FF072
:102490004809686BC6F3044619FB060920684FEA31
:1024A000461A0028B4BF40F0804C4FEA804CC9F86F
:1024B00000C02068400044BF4CF00050C9F8000044
:1024C000300694F80CC040EA0C40C9F8040094F8B7
:1024D0000DC0BCF1000F26D040F44010C9F8040034
:1024E000D1F8C0040130C1F8C00405EB0A0101F5C0
:1024F0008351087F40F020000877207BCDE902233C
:1025000001F02AF80330DDE902238010F9B2013727
:10251000814210DA04EB810C09EB8101DCF804C084
:10252000C1F808C0F2E705EB0A0101F58351087F05
:102530006CF34510E0E70120E96B04F10C07B040B3
:10254000C1F8D00006F18301204605EB4111C1E935
:10255000002305EB461101F58351083150F804CBF7
:10256000B84241F804CBF9D10088AA44088041F26E
:1025700078014AF801600AF5805A08F003019AF8D8
:102580007C0041F0100120F01F0001438AF87C100C
:10259000002181F3118821462846CDF8008000F003
:1025A00089FF012004B0BDE8F087002069E7000042
:1025B0002DE9F04700F58056044696F86254002D48
:1025C00040F0048190F82030032B40F0948028469E
:1025D0002B462F465FFA80FC944510DA01EBCC0EB7
:1025E00051F83CC0BCF1000F04DBDEF804C0BCF1C4
:1025F000000F02DB01370130ECE70133FBE730204D
:1026000080F31188E06BF3B9D0F8803043F0020317
:10261000C0F880304E23E06B002F6FD1D0F88030AF
:1026200043F00103C0F88030694B6A4A1B6803F12C
:10263000805303F52C539B009342A36340F2B08078
:10264000654800F0E7FE4D2B42D8DFF884814FEA61
:10265000034EDFF88891D8F800C04EEA8C0EC0F81F
:1026600084E00CF1805000F52C508000606203EB98
:102670000C00D4F83CC0C3F14E03C8F80000DCF8ED
:10268000800040F03000CCF880004FF0000CD4F80F
:102690002480E6465FFA8CF08242BCDD01EBC00A82
:1026A00051F83000002810DBDAF804A0BAF1000F6E
:1026B0000BDA09EA00400AF07F0A40EA0A0040F01B
:1026C000084048F82E000EF1010E0CF1010CE1E774
:1026D000836923F00103836100F0A2FE0646E36BE9
:1026E0009B69D90704D500F09BFE831BFA2BF6D912
:1026F000002383F311882846BDE8F087B7EB530F1A
:102700003DD2DFF8CCE04FEA074CDEF800304CEA6F
:10271000830CC0F888C003F1805003EB4703002707
:1027200000F52C50CEF80030BC468000A062E06B73
:10273000D0F8803043F00C03C0F88030D4F828E0A3
:10274000FBB29A427FF770AF51F8330001EBC30838
:102750000028D8F8043001DB002B0EDB20F06040AD
:1027600023F0604340F0005043F000434EF83C003B
:102770000EEBCC000CF1010C43600137E0E78369FC
:1027800023F00103836100F04BFE0646E36B9B6977
:10279000DA07ADD500F044FE831BFA2BF6D9A7E784
:1027A000E26B936923F00103936100F039FE074661
:1027B000E36B9B69DB0705D500F032FEC31BFA2BE8
:1027C000F6D995E7012586F8625491E7002592E74E
:1027D000DC630020FCB50040B86800080000FF077B
:1027E00013B500F580540191606DFFF7C5FC1F28FB
:1027F0000AD920220199606DFFF734FDA0F1200372
:102800005842584102B010BD0020FBE708B5302304
:1028100083F3118800F58050406DFFF781FC0023A1
:1028200083F3118808BD00000022026082814260AB
:10283000826070470022002310B5C0E90023002306
:1028400004460C3020F8043CFFF7EEFF204610BD94
:102850002DE9F0479A4688B00746884691463023CE
:1028600083F3118807F580546846FFF7E3FF606D36
:10287000FFF768FC1F282ED920226946606DFFF7FC
:1028800075FD202827D194F8623423B303AD444664
:1028900005AB2E46083403CE9E4244F8080C44F89B
:1028A000041C3546F5D130682060B388A380DDE98B
:1028B0000023C9E90023BDF80830AAF8003000233E
:1028C00083F3118853464A464146384608B0BDE86E
:1028D000F04700F0B3BD002080F3118808B0BDE8D8
:1028E000F08700002DE9F84F06468846182200219F
:1028F00004303546FFF778F8264B06F5825745F841
:10290000403B2C4620462034FFF794FFA742F9D1E4
:1029100006F580544FF4805306F5A4594FF0000A91
:102920002564002567654FF0000B06F58457E564C4
:10293000C4E91135012384F8503084F85830A7F1E8
:102940001800203747E910ABFFF76EFF47F8285C07
:102950004F45F4D1B8F1010F84F86884A4F86A54A3
:10296000A4F86C54A4F86E5484F87054A4F872540B
:10297000A4F87454A4F8765484F8785402D906481C
:1029800000F048FD054B304653F82830F363BDE8AE
:10299000F88F00BF08690008DC680008F8680008C4
:1029A000044B10B5197804464A1C1A70FFF79AFFB9
:1029B000204610BDD96300202DE9F04300295AD0EC
:1029C0002E4E2F48B6FBF1F481428CBF0A20112015
:1029D000431EB4FBF0F700FB1740DDB220B1022B21
:1029E0001846F5D8002032E07B1EB3F5806F2ED25A
:1029F000C5EBC5084FF47A7308F103044FEAE40EFF
:102A0000C4F3C7040EF10109281B0EFB033E5FFA55
:102A100080FC59FA80F0BEFBF0F0B0F5617F18DC65
:102A200083B2601C5CFA80F07843B6FBF0F0814220
:102A3000D8D1611E0F29D5D80CF1FF310729D1D883
:102A40000120138057801071547182F806C0BDE8D0
:102A5000F08308F1FF34E010C4F3C70400F1010E65
:102A60002D1B00FB03335FFA85FC5EFA85F5B3FB93
:102A7000F5F39BB2D5E70846E9E700BF00B4C4040C
:102A80003F420F0030B50D4B05200D4D1C786C43B7
:102A90008C420ED159780120518099785171D978A2
:102AA0009171197911715B7903EB83035B001380DA
:102AB00030BD013803F10603E8D1F9E74C6900089D
:102AC00040420F0038B540F27772C36B154CC3F823
:102AD000BC200722C36BC3F8C8202268C16B9300D7
:102AE00043F4C023C1F8A03002F1805302F16C011D
:102AF000C56B03F52C53EA3289009B00226041F03C
:102B0000E061094AC362C5F8C01003F5D87103F546
:102B10006A7341639342836302D9044800F07AFCEC
:102B200038BD00BFDC630020FCB50040B868000879
:102B30002DE9F04700F580551F4688B0044695F80A
:102B4000683489469046022B04D90026304608B0E6
:102B5000BDE8F087A74A52F8231009B942F82300CC
:102B6000A548C4F81C90017884F82070C9B93023B6
:102B700083F31188A14BD3F8EC2042F48072C3F8A0
:102B8000EC20D3F8942042F48072C3F89420D3F858
:102B9000942022F48072C3F894200123037081F3FF
:102BA000118895F861347BB9302383F31188944AF6
:102BB00095F86834D35C0BB3012B28D0012385F83A
:102BC0006134002383F31188302383F31188E26B8F
:102BD000936923F01003936100F022FC8246E36BBB
:102BE0009E6916F0080619D000F01AFCA0EB0A0343
:102BF000FA2BF4D9002686F31188A7E703211320C6
:102C000002F090F80321152002F08CF8D6E703219A
:102C1000142002F087F803211620F5E79A6942F0A4
:102C200001029A6100F0FCFB8246E36B9A69D007CF
:102C300006D400F0F5FBA0EB0A03FA2BF5D9D9E78F
:102C40009A694FF0000A42F002029A61E36BC3F8FE
:102C500054A08AF31188686DFFF762FA20220021E0
:102C60006846FEF7C1FE02A8FFF7DEFD04F58353B8
:102C70006A460DF1180E3344CDF818A09446083377
:102C8000BCE80300F44543F8080C43F8041C624612
:102C9000F4D1DCF8000020361860B6F5806F9CF89F
:102CA00004201A71DAD1002304F5A35249462046C4
:102CB0000A3285F8603485F86334FFF77DFE0646F6
:102CC00090B9E26B936923F00103936100F0A8FBD4
:102CD0000546E36B9B69D9077FF537AF00F0A0FB92
:102CE000431BFA2BF5D930E795F86E34C5F87C9480
:102CF000591E95F86F34E26B013B1B0243EA4163B6
:102D000095F8701401390B43B5F86C14013943EA96
:102D10000143D361B8F1000F36D004F5A352414608
:102D200020461232FFF7AEFE90B9E26B936923F0B2
:102D30000103936100F074FB0546E36B9B69DA07BE
:102D40007FF503AF00F06CFB431BFA2BF5D9FCE6D3
:102D500095F87724C5F88084511E95F87824E36BA4
:102D6000013A120142EA012295F8761401390A4328
:102D7000B5F87414013942EA014242F40002DA6003
:102D80004FF42062E36B9A64E36B4FF00008204637
:102D9000C3F8BC80FFF796FE85F869846FF0404267
:102DA000E36B1A65174AE36B5A654FF00222E36B37
:102DB0009A654FF0FF32E36BC3F8E0200322E36B28
:102DC0009742DA653FF4C2AEE26B936923F00103E8
:102DD000936100F025FB0746E36B9B69DB0705D594
:102DE00000F01EFBC31BFA2BF6D9AEE6012385F8D3
:102DF0006234ABE6D0630020D86300200044025860
:102E0000F0680008550200022DE9F04F00F5A557C3
:102E10008BB00546904699464FF0000B41F2780A78
:102E20001037EB6BD3F8D83023FA0BF3DC0753D50C
:102E300005EB4B114FEA4B1251440B7918074BD459
:102E400005F58056D6F894340133C6F89434C7E9B2
:102E500000890B79990605EB020148BFD6F8C43406
:102E6000514444BF0133C6F8C4340B7943F008031E
:102E70000B71DB0725D596F8633413B305F583543E
:102E800002A80192FFF7D6FC0834019A05AB14445E
:102E900004F1080C2068083454F8041C1A466445F0
:102EA00003C21346F6D1206802A910602846A28802
:102EB0009A800123ADF810302B68CDE902891B6C94
:102EC0009847D6F8B834D6F864040133C6F8B83455
:102ED00010B103681B6998470BF1010BBBF1200F80
:102EE0009FD10BB0BDE8F08F2DE9F04F0F468DB0AC
:102EF000044600F097FA82468946002F5BD1E36BC7
:102F0000D3F8A02012F4FE0F03D100200DB0BDE8CD
:102F1000F08FD3F8A420920141BF04F58051D1F87D
:102F2000A8240132C1F8A824D3F8A4205606ECD076
:102F3000D3F8A450E66AC5F305254823E8464FF0C8
:102F4000000B03FB05664046FFF76EFC326851003C
:102F50004ABF22F06043C2F38A4343F00043920029
:102F600048BF43F080430093736813F400131BBF02
:102F7000012304F580528DF80D308DF80D301EBF01
:102F8000D2F8C8340133C2F8C834F38803F00F0311
:102F90008DF80C309DF80C0000F0DEFA5FFA8BF330
:102FA000984225D9F2180CA90BF1010B127A0B44A7
:102FB00003F82C2CEEE7012FA7D1E36BD3F8B02058
:102FC00012F4FE0FA1D0D3F8B420950141BF04F54F
:102FD0008051D1F8A8240132C1F8A824D3F8B42034
:102FE000500692D0D3F8B450266BC5F30525A4E75C
:102FF000EFB9E36BC3F8A85004A807ADFFF71AFCBC
:1030000098E80F0007C52B800023204604A9ADF8DF
:103010001830236804F580541B6CCDE904A9984747
:1030200058B1D4F8A0340133C4F8A0346EE7012FAE
:10303000E2D1E36BC3F8B850DEE7D4F8A434012042
:103040000133C4F8A43461E72DE9F04105460F4689
:1030500000F58054012639462846FFF745FF10B198
:1030600084F86364F7E7D4F8B834D4F8640401331F
:10307000C4F8B83420B10368BDE8F0411B691847B3
:10308000BDE8F081C36BF0B51A6C12F47F0F2BD042
:103090001B6C00F5805441F278054FF0010CC4F828
:1030A000BC340023471900EB43125E012A44117916
:1030B00011F0020F15D0490713D4B959C66B0CFA99
:1030C00001F1D6F8CCE011EA0E0F0AD0C6F8D41000
:1030D000117941F004011171D4F89C240132C4F833
:1030E0009C240133202BDED1F0BD00002B4B70B5AA
:1030F0001E561B5C012B30D8294D2A4A55F8233027
:1031000052F8264013B349B3236D9A0510D54FF4F6
:103110000073236500F086F950EA01020B4602D0E5
:10312000013861F10003024655F82600FFF76CFEF6
:10313000236D9B012CD54FF0007255F82630226587
:1031400003F58053012283F8692421E001232365DC
:10315000102323654FF48053236570BD236DDA0778
:1031600002D4236D5B0706D50523002155F8260000
:103170002365FFF769FF236DD80602D4236D590636
:1031800006D55023012155F826002365FFF75CFF83
:1031900055F82600BDE87040FFF774BFF4680008DA
:1031A000D0630020F868000808B5302383F3118845
:1031B000FFF768FF002383F3118808BDC36BD3F8C2
:1031C000C00010F07C5005D0D3F8C40080F400108B
:1031D000C0F340507047000008B5302383F31188D6
:1031E00000F58050406DFEF7ADFF002383F311889A
:1031F00043090CBF0120002008BD000000F58053EA
:1032000093F8692462B1C16B8A6922F001028A6174
:10321000D3F8AC240132C3F8AC24002283F869242B
:10322000704700002DE9F743302181F31188002514
:1032300000F5835141F2780E4FF0010800F5805CF3
:1032400000EB45147444267977071CD4F6061AD58A
:103250008E69D0F83C9008FA06F6D9F8CC703E4258
:1032600011D04F6801970F689742019F9F410AD282
:10327000C9F8D460267946F004062671DCF8984433
:103280000134CCF8984401352031202DD8D10023C9
:1032900083F3118803B0BDE8F0830000F8B51E4643
:1032A00000230F46054613701446FFF795FF80F084
:1032B000010038701EB12846FFF780FF2070F8BD6E
:1032C0002DE9F04F85B099460D468046164691F897
:1032D00000B0DDE90EA302931378019300F0A2F889
:1032E0002B7804460F4613B93378002B41D0224681
:1032F0003B464046FFF796FFFFF756FFFFF77EFF7E
:103300004B4632462946FFF7C9FF2B7833B1BBF154
:10331000000F03D0012005B0BDE8F08F337813B162
:10332000019B002BF6D108F5805303935445029B73
:1033300077EB03031DD2039BD3F86404C8B1036881
:10334000AAEB04011B6898474B4632462946404683
:10335000FFF7A4FF2B7813B1BBF1000FDAD133785C
:1033600013B1019B002BD5D100F05CF804460F4649
:10337000DCE70020CFE70000002108B50846FFF792
:10338000B5FEBDE8084001F0BFB8000008B5012156
:103390000020FFF7ABFEBDE8084001F0B5B8000023
:1033A00008B500210120FFF7A1FEBDE8084001F0AB
:1033B000ABB80000012108B50846FFF797FEBDE84D
:1033C000084001F0A1B8000000B59BB0EFF30981FF
:1033D00068226846FEF7F6FAEFF30583014B9B6B14
:1033E000FEE700BF00ED00E008B5FFF7EDFF0000CD
:1033F00000B59BB0EFF3098168226846FEF7E2FA58
:10340000EFF30583014B5B6BFEE700BF00ED00E0CF
:10341000FEE700000FB408B5029801F037FFFEE7A1
:1034200002F022BB02F004BB0139C9B202299EBFDF
:1034300000EBC1000023C0E901337047F8B51B88D9
:1034400005460E465B0715D4044600F11807BC423A
:1034500010D0636853B12B682846DB6B9847A3688C
:10346000C1B23246606898470834F0E7A368002B81
:10347000F1D1F9E70120F8BD73B56C4684E8060088
:10348000014600224E68D5B26EB98E685EB900EB77
:10349000C2000135021D94E8030082E80300012008
:1034A0001D7002B070BD01320831032AEAD100203C
:1034B000F7E700002DE9F04F89B004460E460546B7
:1034C000BDF8487000F118084FF000094FF0000AED
:1034D00007F004074FF0000BA84539D06B680BB913
:1034E000AB684BB157B923682046DB6B9847AB6894
:1034F000C1B23246686898470835EDE7B9F1000F68
:10350000FAD1334603AA06F1080EADF80890CDE9CA
:1035100000AB1868083353F8041C94467345ACE8B4
:1035200003006246F5D118684FF00109CCF800009D
:103530009B88ACF80430FFF775FF0423ADF8083022
:103540002368CDE900011B6C694620469847D3E704
:10355000012009B0BDE8F08F082817D909280CD040
:103560000A280CD00B280CD00C280CD00D280CD01D
:103570000E2814BF4020302070470C2070471020C8
:1035800070471420704718207047202070470000B3
:103590002DE9F041456A15B94162BDE8F0814B68FB
:1035A000AC4623F06047C3F38A464FEAD37EC3F3A9
:1035B000807816EA230638BF3E462B465A68BEEB93
:1035C000D27F22F060440AD0002A18DAA40CB44258
:1035D00017D19D420FD10D60DEE71346EEE7A742FB
:1035E00007D102F08044C2F3807242450BD054B13F
:1035F000EFE708D2EDE7CCF800100B60CDE7B4425E
:1036000001D0B442E5D81A689C46002AE5D1196079
:10361000C3E700002DE9F047089D01F0070400EB27
:10362000D1004FF47F494FEAD508224405F0070541
:10363000944201D1BDE8F08704F0070705F0070ABE
:10364000111B08EBD50E57453E4613F80EC038BF88
:103650005646C6F108068E4228BF0E46E108415C78
:1036600034443544B94029FA06F721FA0AF1FFB289
:103670008CEA010147FA0AF739408CEA010C03F899
:103680000EC0D5E780EA0120082341F2210201B2F1
:10369000013B4000002980B2B8BF504013F0FF0347
:1036A000F5D1704738B50C468D18A54200D138BD0C
:1036B00014F8011BFFF7E6FFF7E7000042684AB184
:1036C000136881894360438901339BB299424381E6
:1036D00038BF83811046704770B588B004462022F9
:1036E0000D4668460021FEF77FF920460495FFF756
:1036F000E5FF024660B16B46054608AE1C4608353C
:1037000003CCB44245F8080C45F8041C2346F5D117
:10371000104608B070BD0000082817D909280CD041
:103720000A280CD00B280CD00C280CD00D280CD05B
:103730000E2814BF4020302070470C207047102006
:1037400070471420704718207047202070470000F1
:10375000082817D90C280CD910280CD914280CD9F2
:1037600018280CD920280CD930288CBF0F200E2007
:103770007047092070470A2070470B2070470C20C3
:1037800070470D20704700002DE9F843078C044670
:10379000072F1ED900254FF6FF73D0E90298C5F117
:1037A0002006A5F1200029FA05F1083508FA06F6E9
:1037B00028FA00F0314301431846C9B2FFF762FF0F
:1037C000402D0346EBD13A46E169BDE8F843FFF7E7
:1037D00069BF4FF6FF70BDE8F883000010B54B6875
:1037E00023B9CA8A63F30902CA8210BD04691A6840
:1037F0001C600361C38A013BC3824A60EFE700009B
:103800002DE9F84F1D46CB8A0F468146C3F30901C7
:10381000924605290B4630D00020AAB207F11A04BF
:103820009EB21FFA80F8042E0FD8904503F10103D1
:1038300006D30A44FB8A62F309030120FB821AE0E3
:103840001AF800600130E654EAE79045F1D2A1F1A0
:10385000050B1C237C68BBFBF3F203FB12BB1FFAB6
:103860008BF6002C45D14846FFF728FF044638B9AF
:1038700078606FF00200BDE8F88F4FF00008E6E7CF
:10388000002606607860ADB24FF0000B454510D9B8
:103890000AEB0803221D13F8011B08F101089155DA
:1038A000B1B21FFA88F81B292BD0454506F1010655
:1038B000F1D8FB8AC3F30902154465F30903BCE799
:1038C00001321C4692B22368002BF9D16B1F0B44C6
:1038D0001C21B3FBF1F301339BB29A42D3D2BBF16B
:1038E000000FD0D14846FFF7E9FE20B9C4F800B078
:1038F000BFE70122E7E7C0F800B05E46206004465B
:10390000C1E74545D5D94846FFF7D8FE08B920603C
:10391000AFE7C0F800B0002620600446B6E700001C
:103920002DE9F04F1C46074688462DED028B83B0EB
:103930005B690192002B00F0A780238C2BB1E26918
:10394000002A00F0A180072B35D807F10C00FFF703
:10395000B5FE054638B96FF00205284603B0BDEC48
:10396000028BBDE8F08F14220021FEF73DF8228C77
:10397000E16905F10800FEF725F8208C48F00041C8
:10398000013080B2FFF7E4FEFFF7C6FE013880B2D7
:1039900020840130287438466369228C1B782A44BD
:1039A00003F01F0363F03F03137269602946FFF7BA
:1039B000EFFD0125D1E702330722C18A9BB206330E
:1039C000B3FBF2F3828A9BB2521A92B29342C2D8EC
:1039D0004FF0000900F10C034FF0800A4E464D46AF
:1039E00008EE103A18EE100AFFF768FE834600282A
:1039F000B1D014220021FDF7F7FF002E3AD1019B30
:103A00000222ABF808300BF1080E1FFA82FC218C61
:103A10000CF10100BCF1060F80B201D88E422BD30D
:103A2000FFF796FE8E4208BF4FF0400AFFF774FE84
:103A300062690138013512781BFA80F1013002F019
:103A40001F022DB242EA491289F001094AEA020A2C
:103A500048F0004281F808A059468BF8100038461B
:103A6000CBF804204FF0000AFFF792FD238CB342FD
:103A7000B8D172E70022C6E7E169895D01360EF828
:103A80000210B6B20132C0E76FF0010565E7000031
:103A9000F8B515460E463022002104461F46FDF7B4
:103AA000A3FF069BB5F5001FA760636004F110003B
:103AB000079B34BF6A094FF6FF72E661A3620023D9
:103AC00097B29A4206D800230360A782E382238339
:103AD000E360F8BD0660013330462036F1E70000B0
:103AE00003781BB94BB2002BC8BF017070470000B0
:103AF00000787047F8B50C46C969074611B9238CA0
:103B0000002B37D1257E1F2D34D8387828BB228C46
:103B1000072A2CD8268A36F003032BD14FF6FF70E4
:103B2000FFF7C0FD20F0010031024FF6FF724004A4
:103B300041EA0561400C41EA4025234629463846C2
:103B4000FFF7EEFE002807DD626913780133DBB270
:103B50001F2B88BF00231370F8BD218A2D0645EA6C
:103B6000012505432046FFF70FFE0246E5E76FF00B
:103B70000300F1E76FF00100EEE7000070B58AB0D6
:103B8000044616460021282268461D46FDF72CFFF4
:103B9000BDF8383069462046ADF810300F9B0593CC
:103BA0009DF840308DF81830119B0793BDF84830D0
:103BB000CDE90265ADF82030FFF79CFF0AB070BD7B
:103BC0002DE9F041D36905460C4616460BB9138C16
:103BD0005BBB377E1F2F28D895F80080B8F1000F07
:103BE00026D03046FFF7D0FD337821020246284622
:103BF00041EAC331338A41EA080141EA076141EAF7
:103C00000341334641F08001FFF78AFE00280ADDB8
:103C10003378012B07D1726913780133DBB21F2B84
:103C200088BF00231370BDE8F0816FF00100FAE750
:103C30006FF00300F7E70000F0B58BB004460D46C7
:103C400017460021282268461E46FDF7CDFE9DF846
:103C50004C30294620465A1E534253416A468DF83D
:103C600000309DF84030ADF81030119B05939DF861
:103C700048308DF81830149B0793BDF85430CDE9C7
:103C80000276ADF82030FFF79BFF0BB0F0BD0000CF
:103C9000406A00B104307047436A1A6842620269A0
:103CA0001A600361C38A013BC38270472DE9F0416A
:103CB000D0F8208014461D46184E4146002709B909
:103CC000BDE8F081D1E90223A21A65EB0303964215
:103CD00077EB03031ED2036A8B420DD1FFF77EFD03
:103CE000036A1B68036203690B60C38A0161013BBD
:103CF000016AC3828846E2E7FFF770FD0B68C8F8E7
:103D0000003003690B60C38A0161013BC382D8F8AC
:103D10000010D4E788460968D1E700BF80841E0000
:103D20002DE9F04F8BB00D4614469B46DDF85090C0
:103D30008046002800F01881B9F1000F00F01481CE
:103D4000531E3F2B00F21081012A03D1BBF1000F5B
:103D500040F00A810023CDE90833B8F81430B5EB00
:103D6000C30F4FEAC30703D300200BB0BDE8F08FA9
:103D70002B199F42D8F80C3036BF7F1B2746FFB265
:103D80001BB9D8F81030002B7AD0272D4DD8C5F1AB
:103D9000280600232946B742009308ABD8F808004C
:103DA0002CBFF6B23E46A7EB060A354432465FFA10
:103DB0008AFAFFF72FFCB8F81430282103F10053DA
:103DC000053BDB000493D8F80C300393039B13B13D
:103DD000BAF1000F2CD1D8F8100040B1BAF1000FA1
:103DE00005D008AB5246691A0096FFF713FC38B2AB
:103DF000002FB9D066070AD00AAB624203EBD401A8
:103E000002F0070211F8083C134101F8083C082CA5
:103E10003DD9102C40F2B580202C40F2B780BBF188
:103E2000000F00F09C80082335E0BA460026C2E768
:103E3000049BE02B28BFE02306930B44AB42059381
:103E400015D95A1B0398691A0096924508AB00F1E0
:103E5000040034BF5246D2B20792FFF7DBFB079A49
:103E60001644AAEB020A1544F6B25FFA8AFA049BDA
:103E7000069A05999B1A0493039B1B680393A5E775
:103E800000933A4608AB2946D8F80800ADE7BBF1E5
:103E9000000F13D00123B4EBC30F6BD0082C12D842
:103EA0009DF82030621E23FA02F2D50706D54FF0A6
:103EB000FF3202FA04F423438DF820309DF82030BD
:103EC00089F8003051E7102C12D8BDF82030621E5E
:103ED00023FA02F2D10706D54FF0FF3202FA04F4BA
:103EE0002343ADF82030BDF82030A9F800303CE77E
:103EF000202C0FD80899631E21FA03F3DA0705D5A1
:103F00004FF0FF3202FA04F40C430894089BC9F8FE
:103F100000302AE7402C2AD0611EC4F12102A4F10E
:103F20002103DDE9086526FA01F105FA02F225FA16
:103F300003F311431943CB0711D50122A4F1200348
:103F4000C4F1200102FA03F322FA01F1A2400B436B
:103F5000524263EB430332432B43CDE90823DDE9AF
:103F60000823C9E9002300E76FF00100FDE66FF0C8
:103F70000800FAE6082CA1D9102CB4D9202CEED8D0
:103F8000C4E7BBF1000FAED0022384E7BBF1000F02
:103F9000BCD004237FE70000012A30B5144638BFA7
:103FA000012485B00025402C28BF4024012ACDE9FA
:103FB000025518D81B788DF8083063070AD004AB77
:103FC000624203EBD40502F0070215F8083C934067
:103FD00005F8083C034600912246002102A8FFF79D
:103FE00019FB05B030BD082AE4D9102A03D81B8874
:103FF000ADF80830E1E7202A95BF1B68D3E900231C
:104000000293CDE90223D8E710B5CB681BB98B60CA
:104010000B618B8210BD04691A681C600361C38A3E
:10402000013BC382CA60F0E703064CBFC0F3C03057
:104030000220704708B50246FFF7F6FF022806D1B6
:104040005306C2F30F2001D100F0030008BDC2F3F4
:104050000740FBE72DE9F04F93B004460D46CDE94C
:1040600003230A681046FFF7DFFF0228824614BFC9
:10407000C2F306260026002A80F2F88112F0C04919
:1040800040F0F481097B002900F0F081022803D080
:104090002378B34240F0ED81C2F304631046294413
:1040A000069302F07F030593FFF7C4FF059B0022F0
:1040B00083464FEA8348002348EA0A4848EA4668AC
:1040C000CE78CDE90823F30948EA0008029368D0C6
:1040D000059B024608A92046009353466768B847E7
:1040E000002800F0C981276A4FB9414604F10C004D
:1040F000FFF7F2FA074690B96FF0020055E03B690E
:1041000098450DD03F68002FF9D1414604F10C00CD
:10411000FFF7E2FA07460028EED0236A3B602762E9
:1041200097F817C006F01F08CCF3840CACEB08001E
:10413000A8EB0C031FFA80FE0028B8BF0EF1200088
:104140001FFA83FEB8BF00B2002B0793B8BF0EF171
:104150002003D7E90221BCBF1BB2079352EA010337
:1041600038D0039B4FF0000CDFF81CE39A1A049B35
:1041700063EB010196457CEB01032BD36B7B97F836
:104180001AE0734519D1029B002B78D0012821DC5D
:104190007868F8B9DFF8ECC2944570EB010316D3E8
:1041A00037E0276A27B96FF00C0013B0BDE8F08F35
:1041B0003B699845B4D03F68F4E7B24890427CEB45
:1041C000010301D30020F0E7029B002BFAD0079BEC
:1041D0000F2B17DCFA7DB3003946204602F00302AC
:1041E00003F07C031343FB75FFF7F8FA6B7BBB7698
:1041F000029B3BB9FB7DC3F38402013262F3860369
:10420000FB75D0E76A7BBB7E9A42DBD1029B002B19
:1042100035D0B309022B32D0039B142200210DA804
:10422000BB60049BFB60FDF7DFFB039B0AA92046F4
:104230000A93049BADF83EB00B932B1D8DF840A064
:104240000C932B7B8DF84180013BDBB2ADF83C3009
:10425000069B8DF84230059B8DF8433094F82C3046
:1042600083F001038DF84430A3689847FB7DC3F3C6
:104270008403013303F01F039B02FB82A2E7FB7D53
:10428000C6F34012B2EBD31F40F0F980C3F38403AE
:10429000434540F0FB80029AB6092B7B002A52D09E
:1042A00016F0010661D1032B40F2F380039B3946DF
:1042B00004F10C00BB60049BFB60FB8A66F30903FE
:1042C000AE1DFB8232462B7B033BDBB2FFF798FA35
:1042D00000280CDA39462046FFF780FAFB7DC3F34D
:1042E0008403013303F01F039B02FB8204E7AB88C6
:1042F000DDE908843B834FF6FF73C9F12000A9F183
:10430000200228FA09F109F1080904FA00F024FA58
:1043100002F2014318461143C9B2FFF7B3F9B9F1EC
:10432000400F0346E9D1B88231462A7B033AD2B224
:10433000FFF7B8F9FB7DB882DA43C2F3C01262F32B
:10434000C713FB753EE786B92E1D013B394604F1C4
:104350000C00DBB23246FFF753FA0028BADB2A7BA7
:104360003146B88A013AD2B2E2E7F98A013BC1F399
:104370000901DAB204295BD8281D002307F11B06C6
:104380009A4208D910F801CB013306F801C0013177
:10439000DBB20529F4D1039993420A9138BF043363
:1043A00004992CBF002355FA83F30B9107F11B01ED
:1043B0000C9179680E930D91291DFB8AADF83EB0E2
:1043C000C3F309038DF840A08DF841801A44069B81
:1043D0008DF84230059BADF83C208DF8433094F8C1
:1043E0002C3083F001038DF844300023B88A7B60C1
:1043F0002A7B013AFFF756F93B8BB882834203D1FF
:10440000A3680AA92046984720460AA9FFF7FCFDA1
:10441000FB7DBA8AC3F38403013303F01F039B02BD
:10442000FB823B8B9A420CBF00206FF01000BCE671
:104430007B68002BAFD0052001E01C3033461E689E
:10444000002EFAD1091A2E1D081D184401EB090C83
:104450005FFA89F3BCF11B0F9DD89A429BD916F8DD
:10446000013B09F1010900F8013BEFE76FF009009A
:104470009BE66FF00A0098E66FF00B0095E66FF090
:104480000D0092E640420F0080841E006FF00E0087
:104490008BE66FF00F0088E6EFF309830549683378
:1044A0004A6B22F001024A6383F30988002383F3F5
:1044B0001188704700EF00E0302080F3118862B669
:1044C0000D4B0E4AD96821F4E0610904090C0A4336
:1044D0000B49DA60D3F8FC2042F08072C3F8FC206C
:1044E000084AC2F8B01F116841F001011160202292
:1044F000DA7783F82200704700ED00E00003FA0548
:1045000055CEACC5001000E0302310B583F3118800
:104510000E4B5B6813F4006314D0F1EE103AEFF326
:1045200009844FF08073683CE361094BDB6B2366C1
:1045300084F3098800F070FE10B1064BA36110BD32
:10454000054BFBE783F31188F9E700BF00ED00E0BE
:1045500000EF00E03F0400084204000808B5074BE4
:10456000074A196801F03D01996053680BB19068E2
:104570009847BDE80840FFF7C7BF00BF00000240F2
:10458000E463002008B5084B1968890901F03D0172
:104590008A019A60054AD3680BB110699847BDE853
:1045A0000840FFF7B1BF00BF00000240E4630020F5
:1045B00008B5084B1968090C01F03D010A049A601E
:1045C000054A53690BB190699847BDE80840FFF769
:1045D0009BBF00BF00000240E463002008B5084B09
:1045E0001968890D01F03D018A059A60054AD36971
:1045F0000BB1106A9847BDE80840FFF785BF00BFC0
:1046000000000240E463002008B5074B074A5968E0
:1046100001F03D01D960536A0BB1906A9847BDE83B
:104620000840FFF771BF00BF00000240E4630020B4
:1046300008B5084B5968890901F03D018A01DA6023
:10464000054AD36A0BB1106B9847BDE80840FFF7E5
:104650005BBF00BF00000240E463002008B5084BC8
:104660005968090C01F03D010A04DA60054A536BF0
:104670000BB1906B9847BDE80840FFF745BF00BFFE
:1046800000000240E463002008B5084B5968890D1A
:1046900001F03D018A05DA60054AD36B0BB1106C5D
:1046A0009847BDE80840FFF72FBF00BF0000024059
:1046B000E463002008B5074B074A196801F03D0183
:1046C0009960536C0BB1906C9847BDE80840FFF7B8
:1046D0001BBF00BF00040240E463002008B5084B84
:1046E0001968890901F03D018A019A60054AD36C75
:1046F0000BB1106D9847BDE80840FFF705BF00BF3C
:1047000000040240E463002008B5084B1968090C56
:1047100001F03D010A049A60054A536D0BB1906D9A
:104720009847BDE80840FFF7EFBE00BF0004024015
:10473000E463002008B5084B1968890D01F03D01BC
:104740008A059A60054AD36D0BB1106E9847BDE893
:104750000840FFF7D9BE00BF00040240E463002018
:1047600008B5074B074A596801F03D01D960536EFF
:104770000BB1906E9847BDE80840FFF7C5BE00BF7B
:1047800000040240E463002008B5084B5968890919
:1047900001F03D018A01DA60054AD36E0BB1106F5A
:1047A0009847BDE80840FFF7AFBE00BF00040240D5
:1047B000E463002008B5084B5968090C01F03D017D
:1047C0000A04DA60054A536F0BB1906F9847BDE851
:1047D0000840FFF799BE00BF00040240E4630020D8
:1047E00008B5084B5968890D01F03D018A05DA606A
:1047F000054AD36F13B1D2F880009847BDE808404E
:10480000FFF782BE00040240E463002000230C494D
:1048100010B51A460B4C0B6054F82300026001EBF4
:10482000430004334260402BF6D1074A4FF0FF3378
:104830009360D360C2F80834C2F80C3410BD00BFD6
:10484000E46300206C690008000002400F28F8B5FE
:1048500010D9102810D0112811D0122808D10F24F7
:104860000720DFF8B4E00126DEF80050A04208D9A6
:10487000002649E00446F4E70F240020F1E707246E
:10488000FBE706FA00F73D4240D1214C4FEA001CFD
:104890003D4304EB00160EEBC000CEF80050C0E91B
:1048A0000123FBB24BB11B48836B43F001038363CD
:1048B000036E43F001030366036E17F47F4F09D0C4
:1048C0001448836B43F002038363036E43F00203D7
:1048D0000366036E54F80C00036823F01F030360A3
:1048E000056815F00105FBD104EB0C033D2493F89A
:1048F0000CC05F6804FA0CF43C602124056044613C
:1049000012B1987B00F00EFA3046F8BD0130ADE7E9
:104910006C69000800450258E463002010B530249B
:1049200084F31188FFF792FF002383F3118810BDF1
:1049300010B50446807B00F00BFA01231049627B1E
:1049400003FA02F20B6823EA0203DAB20B604AB9F7
:104950000C4A916B21F001019163116E21F001016C
:104960001166126E13F47F4F09D1064B9A6B22F039
:1049700002029A631A6E22F002021A661B6E10BDC2
:10498000E46300200045025808B5302383F3118802
:10499000FFF7CEFF002383F3118808BD0023054AEB
:1049A00019460133102BC2E9001102F10802F8D1B7
:1049B000704700BF686400202DE9F74F02F0030A3A
:1049C000C2F3C313C2F38009C2F3C108C2F3411E8C
:1049D000574600224FF00F0B0193CB0733D502F05F
:1049E0000703019C012556009B00BAF1020F05FA4E
:1049F00002F504FA03FC44680BFA03F324EA050405
:104A00006FEA030344EA090444604FF00304856835
:104A100004FA06F625EA06056FEA060445EA0805E3
:104A20008560C56825EA060545EA0E05C5601BD107
:104A3000072A13D8056A2B4043EA0C030362036874
:104A40001C403C430460490822D04FEA4909013226
:104A50004FEA88084FEA8E0EBF00BEE7456A2B403A
:104A600043EA0C034362EAE70568072A04EA0504FF
:104A700044EA0704046005D8046A234043EA0C03AF
:104A80000362E0E7446A234043EA0C034362DAE747
:104A900003B0BDE8F08F0000026843681143016075
:104AA00003B1184770470000024A136843F0C0037F
:104AB0001360704700100140024A136843F0C003BE
:104AC00013607047007C004037B51A4C1A4D2046E1
:104AD00000F0E8FA04F11400009400234FF400728F
:104AE000164900F0A5F94FF40072154904F1380099
:104AF0000094144B00F01EFA134BC4E91735134C05
:104B0000204600F0CFFA04F1140000234FF40072A5
:104B10000F49009400F08CF90E4B4FF400720E49CF
:104B200004F13800009400F005FA0C4BC4E9173585
:104B300003B030BDE864002000E1F505C065002049
:104B4000C0690020A94A00080010014054650020F7
:104B5000C0670020B94A0008C06B0020007C0040FC
:104B6000037C30B5284C002918BF0C46012B0CD112
:104B7000264B984236D1264B1A6D42F010021A6528
:104B80009A6F42F010029A679B6F2268036EC16DA4
:104B900003EB52038466B3FBF2F36268150442BF71
:104BA00023F0070503F0070343EA4503CB60A3683E
:104BB00043F040034B60E36843F001038B6042F431
:104BC000967343F001030B604FF0FF330B62510506
:104BD00005D512F0102213D0B2F1805F12D080F808
:104BE000643030BD0B4B9842CFD1094B9A6C42F0E8
:104BF00000429A641A6F42F000421A671B6FC4E7C2
:104C00007F23ECE73F23EAE76C6A0008E8640020B2
:104C100000450258546500202DE9F047C66D054651
:104C20003768F469210734621AD014F0080118BFFC
:104C30004FF48071E20748BF41F02001A3074FF015
:104C4000300348BF41F04001600748BF41F0800198
:104C500083F31188281DFFF71FFF002383F31188BA
:104C6000E2050AD5302383F311884FF48061281DB3
:104C7000FFF712FF002383F311884FF030094FF044
:104C8000000A14F0200838D13B0616D54FF0300941
:104C900005F1380A200610D589F31188504600F036
:104CA0007DF9002836DA0821281DFFF7F5FE27F0E8
:104CB00080033360002383F31188790614D56206DC
:104CC00012D5302383F31188D5E913239A4208D1F2
:104CD0002B6C33B127F040071021281DFFF7DCFEB5
:104CE0003760002383F31188E30618D5AA6E136991
:104CF000ABB15069BDE8F047184789F31188736A72
:104D0000284695F86410194000F0E6F98AF31188F6
:104D1000F469B6E7B06288F31188F469BAE7BDE8D0
:104D2000F0870000090100F16043012203F56143AF
:104D3000C9B283F8001300F01F039A4043099B0097
:104D400003F1604303F56143C3F880211A607047A3
:104D500000F01F0301229A40430900F160409B00CC
:104D600000F5614003F1604303F56143C3F880201F
:104D7000C3F88021002380F800337047F8B515464A
:104D8000826804460B46AA4200D28568A16926695A
:104D9000761AB5420BD218462A46FCF713FEA369D1
:104DA0002B44A3612846A3685B1BA360F8BD0CD904
:104DB000AF1B18463246FCF705FE3A46E168304420
:104DC000FCF700FEE3683B44EBE718462A46FCF795
:104DD000F9FDE368E5E7000083689342F7B5044610
:104DE000154600D28568D4E90460361AB5420BD264
:104DF0002A46FCF7E7FD63692B4463612846A368F4
:104E00005B1BA36003B0F0BD0DD93246AF1B01910F
:104E1000FCF7D8FD01993A46E0683144FCF7D2FD31
:104E2000E3683B44E9E72A46FCF7CCFDE368E4E7A6
:104E300010B50A440024C361029B8460C160026112
:104E40000362C0E90000C0E9051110BD08B5D0E952
:104E50000532934201D1826882B982680132826050
:104E60005A1C426119700021D0E904329A4224BFD1
:104E7000C368436100F076FA002008BD4FF0FF30B0
:104E8000FBE7000070B5302304460E4683F311881B
:104E9000A568A5B1A368A269013BA360531CA361E7
:104EA00015782269934224BFE368A361E3690BB1DB
:104EB00020469847002383F31188284607E03146AF
:104EC000204600F03FFA0028E2DA85F3118870BD31
:104ED0002DE9F74F04460E4617469846D0F81C9029
:104EE0004FF0300A8AF311884FF0000B154665B178
:104EF0002A4631462046FFF741FF034660B9414646
:104F0000204600F01FFA0028F1D0002383F3118817
:104F1000781B03B0BDE8F08FB9F1000F03D001900A
:104F20002046C847019B8BF31188ED1A1E448AF373
:104F30001188DCE7C160C361009B82600362C0E945
:104F400005111144C0E9000001617047F8B504463D
:104F50000D461646302383F31188A768A7B1A368CE
:104F6000013BA36063695A1C62611D70D4E904327D
:104F70009A4224BFE3686361E3690BB12046984716
:104F8000002080F3118807E03146204600F0DAF96E
:104F90000028E2DA87F31188F8BD0000D0E9052384
:104FA00010B59A4201D182687AB982680021013233
:104FB00082605A1C82611C7803699A4224BFC368CC
:104FC000836100F0CFF9204610BD4FF0FF30FBE7C2
:104FD0002DE9F74F04460E4617469846D0F81C9028
:104FE0004FF0300A8AF311884FF0000B154665B177
:104FF0002A4631462046FFF7EFFE034660B9414698
:10500000204600F09FF90028F1D0002383F3118897
:10501000781B03B0BDE8F08FB9F1000F03D0019009
:105020002046C847019B8BF31188ED1A1E448AF372
:105030001188DCE7026843681143016003B1184737
:10504000704700001430FFF743BF00004FF0FF33FC
:105050001430FFF73DBF00003830FFF7B9BF000044
:105060004FF0FF333830FFF7B3BF00001430FFF7C5
:1050700009BF00004FF0FF311430FFF703BF0000FD
:105080003830FFF763BF00004FF0FF323830FFF7D2
:105090005DBF0000012914BF6FF0130000207047AE
:1050A000FFF712BD044B036000234360C0E90233E5
:1050B00001230374704700BF846A000810B53023D1
:1050C000044683F31188FFF74BFD0223002023746D
:1050D00080F3118810BD000038B5C36904460D4641
:1050E0001BB904210844FFF7A5FF294604F1140069
:1050F000FFF7ACFE002806DA201D4FF40061BDE882
:105100003840FFF797BF38BD0023826803750369F5
:105110001B6899689142FBD25A6803604260106034
:105120005860704700238268037503691B6899689B
:105130009142FBD85A680360426010605860704723
:1051400008B50846302383F311880A7D0023052A19
:1051500006D8DFE802F00B050503120E8269136022
:105160004FF0FF338361FFF7CFFF002383F31188F4
:1051700008BD8269936801339360D0E900321360FF
:105180005A60EDE7FFF7C0BF054BD968087518688E
:10519000026853601A600122D8600275FBF73AB9C1
:1051A000C06D00200C4B30B5DD684B1C87B0044649
:1051B0000FD02B46094A684600F066F92046FFF7F3
:1051C000E3FF009B13B1684600F068F9A86907B0D7
:1051D00030BDFFF7D9FFF9E7C06D0020415100084D
:1051E00038B50C4D04468161EB6881689A6891423C
:1051F00003D8BDE83840FFF787BF1846FFF792FF96
:1052000001230146EC6020462375BDE83840FBF7DA
:1052100001B900BFC06D0020044B1A68DB689068BC
:105220009B68984294BF002001207047C06D002009
:10523000084B10B51C68D868226853601A600122B8
:10524000DC602275FFF76EFF01462046BDE8104086
:10525000FBF7E0B8C06D002038B50123084C0025ED
:105260002370656000F0ACFD00F0D2FD05490648F2
:1052700000F0A6FE0223237085F3118838BD00BF1D
:1052800028700020B06A0008C06D002008B572B612
:10529000044B186500F0BEFB00F080FC024B0322BB
:1052A0001A70FEE7C06D00202870002000F02CB9B5
:1052B0008B600223086108468B8270478368A3F1E4
:1052C000840243F8142C026943F8442C426943F8E1
:1052D000402C094A43F8242CC268A3F1200043F86B
:1052E000182C022203F80C2C002203F80B2C034A82
:1052F00043F8102C704700BF2D040008C06D00203B
:1053000008B5FFF7DBFFBDE80840FFF73BBF000033
:10531000024BDB6898610F20FFF736BFC06D00209D
:10532000302383F31188FFF7F3BF000008B501466F
:10533000302383F311880820FFF734FF002383F321
:10534000118808BD064BDB6839B1426818605A60A5
:10535000136043600420FFF725BF4FF0FF30704714
:10536000C06D00200368984206D01A680260506041
:1053700018469961FFF706BF70470000036810B533
:105380009C68A2420CD85C688A600B604C6021600B
:10539000596099688A1A9A604FF0FF33836010BD94
:1053A000121B1B68ECE700000A2938BF0A2170B500
:1053B00004460D460A26601900F0FCFC00F0E4FCEF
:1053C000041BA54203D8751C04462E46F3E70A2E9B
:1053D00004D90120BDE8704000F032BE70BD00006D
:1053E000F8B5144B0D460A2A4FF00A07D96103F1AC
:1053F0001001826038BF0A224160196914460160B9
:1054000048601861A81800F0C5FC00F0BDFC431B03
:105410000646A34206D37C1C28192746354600F0D1
:10542000C9FCF2E70A2F04D90120BDE8F84000F0DA
:1054300007BEF8BDC06D0020F8B506460D4600F069
:10544000A3FC0F4A134653F8107F9F4206D12A4609
:1054500001463046BDE8F840FFF7C2BFD169BB68DE
:10546000441A2C1928BF2C46A34202D92946FFF71B
:105470009BFF224631460348BDE8F840FFF77EBF58
:10548000C06D0020D06D0020C0E90323002310B4BC
:105490005DF8044B4361FFF7CFBF000010B5194C16
:1054A000236998420DD08168D0E9003213605A60B8
:1054B0009A680A449A60002303604FF0FF33A361A7
:1054C00010BD0268234643F8102F5360002202608B
:1054D00022699A4203D1BDE8104000F065BC936890
:1054E00081680B44936000F04FFC2269E169926887
:1054F000441AA242E4D91144BDE81040091AFFF74A
:1055000053BF00BFC06D00202DE9F047DFF8BC801D
:1055100008F110072C4ED8F8105000F035FCD8F8E0
:105520001C40AA68031B9A423ED814444FF000095D
:10553000D5E90032C8F81C4013605A60C5F80090E5
:10554000D8F81030B34201D100F02EFC89F3118855
:10555000D5E9033128469847302383F311886B69D6
:10556000002BD8D000F010FC6A69A0EB0409824639
:105570004A450DD2022000F063FD0022D8F8103019
:10558000B34208D151462846BDE8F047FFF728BF8F
:10559000121A2244F2E712EB09092946384638BFAD
:1055A0004A46FFF7EBFEB5E7D8F81030B34208D013
:1055B0001444C8F81C00211AA960BDE8F047FFF7A1
:1055C000F3BEBDE8F08700BFD06D0020C06D0020A5
:1055D00038B500F0D9FB054AD2E90845031B181974
:1055E00045F10001C2E9080138BD00BFC06D0020CF
:1055F00000207047FEE70000704700004FF0FF30CA
:1056000070470000BFF34F8F044B1A695107FCD15C
:10561000D3F810215207F8D1704700BF0020005284
:1056200008B50D4B1B78ABB9FFF7ECFF0B4BDA68F5
:10563000D10704D50A4A5A6002F188325A60D3F879
:105640000C21D20706D5064AC3F8042102F188329C
:10565000C3F8042108BD00BF3070002000200052B4
:105660002301674508B5114B1B78F3B9104B1A6934
:10567000510703D5DA6842F04002DA60D3F810210E
:10568000520705D5D3F80C2142F04002C3F80C2193
:10569000FFF7B8FF064BDA6842F00102DA60D3F890
:1056A0000C2142F00102C3F80C2108BD307000202B
:1056B000002000520F289ABF00F5806040040020AF
:1056C000704700004FF40030704700001020704712
:1056D0000F2808B50BD8FFF7EDFF00F5003302687F
:1056E000013204D104308342F9D1012008BD0020E9
:1056F000FCE700000F2838B505463FD8FFF782FFCA
:105700001F4CFFF78DFF4FF0FF3307286361C4F88C
:1057100014311DD82361FFF775FF030243F0240302
:10572000E360E36843F08003E36023695A07FCD435
:105730002846FFF767FFFFF7BDFF4FF4003100F089
:1057400009FA2846FFF78EFFBDE83840FFF7C0BFD3
:10575000C4F81031FFF756FFA0F108031B0243F015
:105760002403C4F80C31D4F80C3143F08003C4F89E
:105770000C31D4F810315B07FBD4D9E7002038BDD9
:10578000002000522DE9F84F05460C46104645EA28
:105790000203DE0602D00020BDE8F88F20F01F00D3
:1057A000DFF8BCB0DFF8BCA0FFF73AFF04EB00085D
:1057B000444503D10120FFF755FFEDE7202229469C
:1057C000204601F00BF810B920352034F0E72B46C5
:1057D00005F120021F68791CDDD104339A42F9D10A
:1057E00005F178431B481C4EB3F5801F1B4B38BF97
:1057F000184603F1F80332BFD946D1461E46FFF7DB
:1058000001FF0760A5EB040C336804F11C0143F0B1
:1058100002033360231FD9F8007017F00507FAD18F
:1058200053F8042F8B424CF80320F4D1BFF34F8F71
:10583000FFF7E8FE4FF0FF332022214603602846A1
:10584000336823F00203336000F0C8FF0028BBD0A8
:105850003846B0E7142100520C20005214200052A8
:10586000102000521021005210B5084C237828B1A6
:105870001BB9FFF7D5FE0123237010BD002BFCD010
:105880002070BDE81040FFF7EDBE00BF3070002073
:105890002DE9F04F0D4685B0814658B111F00D0647
:1058A00014BF2022082211F00803019304D0431EE4
:1058B00003426AD0002435E0002E37D009F11F01E1
:1058C00021F01F094FF00108324F05F00403DFF803
:1058D000D0A005EA080BBBF1000F32D07869C007F1
:1058E0002FD408F101080C37B8F1060FF3D19EB997
:1058F000294D4946A819019200F0ACFA0446002847
:105900003AD11836019A782EF3D1494600F0A2FA1E
:105910000446002830D1019A4946204800F09AFAFE
:10592000044668BB204605B0BDE8F08F0029C9D108
:1059300001462846029200F08DFA0446E0B9029A28
:10594000C0E713B178694107CBD5AC0702D57869B8
:105950008007C6D5019911B178690107C1D5182012
:10596000494600FB08A0CDE9022300F073FA044683
:10597000DDE902230028B4D04A460021204601E098
:105980004A460021FCF730F8CCE70246002E95D1BC
:1059900098E700BFBC6A00086470002034700020E3
:1059A0004C7000200121FFF773BF0000F8B5144DC3
:1059B00001241827134E40F2FF3200210120FCF78A
:1059C00013F807FB046001342A6955F80C1F00F036
:1059D0002DFA062CF5D137254FF4C0542046FFF799
:1059E000E1FF014628B122460748BDE8F84000F033
:1059F0001DBAC4EBC404013D4FEAD404EED1F8BD96
:105A0000BC6A00084C7000203470002008B100F01F
:105A100093BA704738B5054D00240334696855F8CA
:105A20000C0B00F0A9F8122CF7D138BDBC6A0008A5
:105A300038B5EFF311859DB9EFF30584C4F308047D
:105A4000302334B183F31188FFF7C2FD85F3118849
:105A500038BD83F31188FFF7BBFD84F3118838BD8F
:105A6000BDE83840FFF7B4BD10B5FFF7E1FF104CBB
:105A7000C008104A002340EA4170C908A0FB04ECAA
:105A8000A0FB020E1CEB0000A1FB044CA1FB0212C8
:105A90005B41001943EB0C0011EB0E0142F10002D7
:105AA000411842F10000090941EA007010BD00BF31
:105AB000CFF753E3A59BC4200244074BD2B210B5E5
:105AC000904200D110BD441C00B253F8200041F8B0
:105AD000040BE0B2F4E700BF504000580E4B30B565
:105AE0001C6F240405D41C6F1C671C6F44F4004415
:105AF0001C670A4C02442368D2B243F480732360CB
:105B0000074B904200D130BD441C51F8045B00B2F9
:105B100043F82050E0B2F4E700440258004802582D
:105B20005040005807B5012201A90020FFF7C4FF2B
:105B3000019803B05DF804FB13B50446FFF7F2FFCC
:105B4000A04205D0012201A900200194FFF7C6FF61
:105B500002B010BD0144BFF34F8F064B884204D3FF
:105B6000BFF34F8FBFF36F8F7047C3F85C022030D5
:105B7000F4E700BF00ED00E00144BFF34F8F064B98
:105B8000884204D3BFF34F8FBFF36F8F7047C3F8C2
:105B900070022030F4E700BF00ED00E07047000025
:105BA000114BDA6952021ED59A69D00704D50F4A03
:105BB0009A6002F144329A600B4BDA69D107FCD447
:105BC0001A6A22F480021A629A6942F002029A6109
:105BD000DA69D207FCD49A6942F001029A61024A5A
:105BE000D369DB07FCD47047002000523B2A190818
:105BF000074B45F255521A6003225A6040F2FF7279
:105C00009A604CF6CC421A600122024B1A7070471F
:105C100000480058E0700020034B1B781BB1034B79
:105C20004AF6AA221A607047E07000200048005827
:105C3000034B1A681AB9034AD2F8D0241A60704785
:105C4000DC70002000400258024B4FF48032C3F851
:105C5000D02470470040025808B5FFF7E9FF024B17
:105C60001868C0F3806008BDDC70002070B5BFF319
:105C70004F8FBFF36F8F1A4A0021C2F85012BFF343
:105C80004F8FBFF36F8F536943F400335361BFF3FA
:105C90004F8FBFF36F8FC2F88410BFF34F8FD2F8CE
:105CA000803043F6E074C3F3C900C3F34E335B01A5
:105CB00003EA0406014646EA81750139C2F86052DA
:105CC000F9D2203B13F1200FF2D1BFF34F8F53696C
:105CD00043F480335361BFF34F8FBFF36F8F70BDB9
:105CE00000ED00E0FEE70000214B2248224A70B59B
:105CF000904237D3214BC11EDA1C121A22F0030244
:105D00008B4238BF00220021FBF76EFE1C4A0023A5
:105D1000C2F88430BFF34F8FD2F8803043F6E0747E
:105D2000C3F3C900C3F34E335B0103EA0406014623
:105D300046EA81750139C2F86C52F9D2203B13F161
:105D4000200FF2D1BFF34F8FBFF36F8FBFF34F8F91
:105D5000BFF36F8F0023C2F85032BFF34F8FBFF3F2
:105D60006F8F70BD53F8041B40F8041BC0E700BFE1
:105D7000846C00080471002004710020047100206C
:105D800000ED00E000F05ABA014B586A704700BFBE
:105D9000000C0040034B002258631A610222DA60B3
:105DA000704700BF000C0040014B0022DA607047D2
:105DB000000C0040014B5863704700BF000C0040CE
:105DC000024B034A1A60034A5A607047E47000208D
:105DD0000871002000000220074B494210B55C68A2
:105DE000201A08401968821A8A4203D3A24201D8B5
:105DF0005A6010BD0020FCE7E470002008B5302395
:105E000083F31188FFF7E8FF002383F3118808BDAF
:105E100004480121044B03600023C0E901330C3026
:105E200000F016B9EC700020FD5D0008CB1D083AAB
:105E300023F00703591A521A012110B4D208002482
:105E4000C0E9004384600C301C605A605DF8044B6C
:105E500000F0FEB82DE9F84F364ECD1D0F46002854
:105E600018BF0646082A4FEAD50538BF082206F1B2
:105E70000C08341D9146404600F006F909F107016F
:105E8000C9F1000E224624686CB9404600F006F9BC
:105E90003368CBB308224946E8009847044698B3D4
:105EA00040E9026730E004EB010CD4F804A00CEAEE
:105EB0000E0C0AF10100ACF1080304EBC00098429B
:105EC000E0D9A0EB0C0CB5EBEC0F4FEAEC0BD9D8FA
:105ED0009C421CD204F10802AB45A3EB02024FEA3C
:105EE000E202626009D9691CED43206803EBC1023C
:105EF0005D44556043F8310022601C465F604046B7
:105F000044F8086B00F0CAF82046BDE8F88FAA45AF
:105F1000216802D111602346EFE7013504EBC50388
:105F200044F8351003F10801401AC010586013609E
:105F3000F1E700BFEC700020F8B550F8043C0446CF
:105F400050F8085CA0F1080607332F1D0C35DB085C
:105F500040F8043C284600F097F83B469F421A68F8
:105F600001D0B34228D20AB1964225D244F8082C77
:105F700054F8042C1E60013254F8081C06EBC200D1
:105F8000814206D14868024444F8042C0A6844F867
:105F9000082C5868411C03EBC1018E4207D154F80C
:105FA000042C013202445A6054F8082C1A60284626
:105FB000BDE8F84000F072B81346CFE7FEE70000F6
:105FC00070B51B4B0025044686B058600E468562AE
:105FD0000163FEF771FA04F11003A560E562C4E9FC
:105FE00004334FF0FF33C4E90044C4E90635FFF73A
:105FF000CBFE2B46024604F134012046C4E90823B7
:1060000080230C4A2565FFF753F901230A4AE06013
:1060100000920375684672680192B268CDE9022366
:10602000064BCDE90435FFF76BF906B070BD00BF34
:1060300028700020046B0008096B0008BD5F000891
:10604000024AD36A1843D062704700BFC06D002077
:10605000C0E90000816070478368013B002B10B5E8
:1060600083600CDA074BDC684368A06120606360E2
:106070001C6044600520FFF787F8A06910BD002070
:10608000FCE700BFC06D002008B5302383F3118802
:10609000FFF7E2FF002383F3118808BD08B5302322
:1060A00083F3118883680133002B836007DC036866
:1060B00000211A68026050601846FFF791F800232B
:1060C00083F3118808BD00004B6843608B688360D0
:1060D000CB68C3600B6943614B6903628B694362A0
:1060E0000B6803607047000008B53C4B40F2FF713D
:1060F0003B48D3F888200A43C3F88820D3F8882087
:1061000022F4FF6222F00702C3F88820D3F8883017
:10611000344B1A6C0A431A649A6E0A439A66324ADE
:106120009B6E1146FFF7D0FF00F5806002F11C0165
:10613000FFF7CAFF00F5806002F13801FFF7C4FFE6
:1061400000F5806002F15401FFF7BEFF00F58060AA
:1061500002F17001FFF7B8FF00F5806002F18C01D9
:10616000FFF7B2FF00F5806002F1A801FFF7ACFF76
:1061700000F5806002F1C401FFF7A6FF00F5806022
:1061800002F1E001FFF7A0FF00F5806002F1FC01E1
:10619000FFF79AFF02F58C7100F58060FFF794FF1E
:1061A00000F00EF9114BD3F8902242F00102C3F82F
:1061B0009022D3F8942242F00102C3F894220522DF
:1061C000C3F898204FF06052C3F89C20084AC3F8E7
:1061D000A020BDE80840FFF7E3BC00BF0044025820
:1061E0000000025800450258106B000800ED00E066
:1061F0001F00080308B500F0CFFAFFF72DF80C4B8D
:10620000DA6B42F04002DA635A6E22F040025A66BC
:106210005B6E084B1A6842F008021A601A6842F076
:1062200004021A60FFF704FDBDE80840FFF7BEBB9B
:106230000045025800180248704700000E4B9A6C47
:1062400042F008029A641A6F42F008021A670B4A79
:106250001B6FD36B43F00803D363C722084B9A62CA
:106260004FF0FF32DA6200229A615A63DA605A60B4
:1062700001225A611A607047004502580010005C04
:10628000000C0040094A08B51169D3680B40D9B227
:106290009B076FEA0101116107D5302383F3118851
:1062A000FFF704F8002383F3118808BD000C0040B9
:1062B000044BDA6B0243DA635A6E104358665B6E26
:1062C000704700BF0045025808B53C4B4FF0FF3106
:1062D000D3F8802062F00042C3F88020D3F88020F9
:1062E00002F00042C3F88020D3F88020D3F8842045
:1062F000C3F88410D3F884200022C3F88420D3F894
:106300008400D86F40F0FF4040F4FF0040F4DF40CD
:1063100040F07F00D867D86F20F0FF4020F4FF00E6
:1063200020F4DF4020F07F00D867D86FD3F88800D2
:106330006FEA40506FEA5050C3F88800D3F88800E5
:10634000C0F30A00C3F88800D3F88800D3F890009F
:10635000C3F89010D3F89000C3F89020D3F89000C1
:10636000D3F89400C3F89410D3F89400C3F89420A1
:10637000D3F89400D3F89800C3F89810D3F8980095
:10638000C3F89820D3F89800D3F88C00C3F88C1089
:10639000D3F88C00C3F88C20D3F88C00D3F89C0081
:1063A000C3F89C10D3F89C10C3F89C20D3F89C3001
:1063B000FEF72CFABDE8084000F0BEB900440258D0
:1063C00008B50122504BC3F80821504B5A6D42F0DA
:1063D00002025A65DA6F42F00202DA670422DB6FCA
:1063E0004B4BDA605A689104FCD54A4A1A60012284
:1063F0009A60494ADA6000221A614FF440429A6179
:10640000434B9A699204FCD51A6842F480721A6070
:10641000424B1A6F12F4407F04D04FF480321A6757
:1064200000221A671A6842F001021A603B4B1A6890
:106430005007FCD500221A611A6912F03802FBD10C
:10644000012119604FF0804159605A67344ADA627D
:10645000344A1A611A6842F480321A602F4B1A6863
:106460009103FCD51A6842F480521A601A689204AB
:10647000FCD52D4A2D499A6200225A63196301F511
:106480007C01DA6301F5E77199635A64284A1A645A
:10649000284ADA621A6842F0A8521A601F4B1A683A
:1064A00002F02852B2F1285FF9D148229A614FF4E4
:1064B0008862DA6140221A621F4ADA641F4A1A654A
:1064C0001F4A5A651F4A9A6532231F4A1360136890
:1064D00003F00F03022BFAD1104A136943F00303B0
:1064E0001361136903F03803182BFAD14FF00050F1
:1064F000FFF7DEFE4FF08040FFF7DAFE4FF000407E
:10650000BDE80840FFF7D4BE0080005100450258A6
:106510000048025800C000F0040000010044025886
:106520000000FF010088900832206000630209012A
:10653000470E0508DD0BBF01200000200000011000
:106540000910E00000010110002000524FF0B0429D
:1065500008B5D2F8883003F00103C2F8883023B1BF
:10656000044A13680BB150689847BDE80840FDF72E
:10657000CBBF00BF686400204FF0B04208B5D2F82E
:10658000883003F00203C2F8883023B1044A9368CC
:106590000BB1D0689847BDE80840FDF7B5BF00BF14
:1065A000686400204FF0B04208B5D2F8883003F09C
:1065B0000403C2F8883023B1044A13690BB150694F
:1065C0009847BDE80840FDF79FBF00BF6864002002
:1065D0004FF0B04208B5D2F8883003F00803C2F893
:1065E000883023B1044A93690BB1D0699847BDE85C
:1065F0000840FDF789BF00BF686400204FF0B0423B
:1066000008B5D2F8883003F01003C2F8883023B1FF
:10661000044A136A0BB1506A9847BDE80840FDF779
:1066200073BF00BF686400204FF0B04310B5D3F8CB
:10663000884004F47872C3F88820A30604D5124A6F
:10664000936A0BB1D06A9847600604D50E4A136B63
:106650000BB1506B9847210604D50B4A936B0BB1D5
:10666000D06B9847E20504D5074A136C0BB1506C08
:106670009847A30504D5044A936C0BB1D06C984796
:10668000BDE81040FDF740BF686400204FF0B04304
:1066900010B5D3F8884004F47C42C3F88820620522
:1066A00004D5164A136D0BB1506D9847230504D5D8
:1066B000124A936D0BB1D06D9847E00404D50F4A90
:1066C000136E0BB1506E9847A10404D50B4A936E1C
:1066D0000BB1D06E9847620404D5084A136F0BB112
:1066E000506F9847230404D5044A936F0BB1D06FC1
:1066F0009847BDE81040FDF707BF00BF6864002061
:1067000008B50348FEF788FABDE80840FDF7FCBE6F
:10671000E864002008B50348FEF77EFABDE80840AB
:10672000FDF7F2BE5465002008B5FFF7ABFDBDE8EC
:106730000840FDF7E9BE0000062108B50846FEF74F
:10674000F1FA06210720FEF7EDFA06210820FEF7F0
:10675000E9FA06210920FEF7E5FA06210A20FEF7EC
:10676000E1FA06211720FEF7DDFA06212820FEF7C0
:10677000D9FA09217A20FEF7D5FA07213220FEF74F
:10678000D1FA0C212520FEF7CDFA0C215320BDE8CB
:106790000840FEF7C7BA000008B5FFF795FDFEF701
:1067A000FDF8FEF77DFCFFF747FDBDE80840FFF769
:1067B000E9BA00000B460146184600F001B8000097
:1067C00010B5054C13462CB10A4601460220AFF322
:1067D000008010BD2046FCE70000000010B5013924
:1067E0000244904201D1002005E0037811F8014FE6
:1067F000A34201D0181B10BD0130F2E72DE9F04192
:10680000A3B1C91A17780144044603F1FF3C8C4236
:10681000204601D9002009E00578BD4204F10104B9
:10682000F5D10CEB0405D618A54201D1BDE8F081E5
:1068300015F8018D16F801EDF045F5D0E7E70000F9
:10684000034611F8012B03F8012B002AF9D17047F8
:10685000636F6D2E6375626570696C6F742E686509
:10686000726534666300000053544D333248373F3D
:106870003F3F0053544D3332483733782F37327807
:106880000053544D3332483734332F3735332F3795
:106890003530000001105A00031059000120580043
:1068A0000320560040A2E4F1646891060041A3E58C
:1068B000F26569920700000043414E464449666113
:1068C00063653A204D6573736167652052414D20C1
:1068D0004F766572666C6F7721000000426164201C
:1068E00043414E496661636520696E6465782E0098
:1068F000000100000001FF0000A0004000A40040D3
:106900000000000000000000312B00089123000867
:10691000C1320008012400080D2400085128000895
:10692000B1250008C9230008CD230008A5230008CD
:106930008D2300080D280008B123000879340008D1
:1069400029340008BD230008E127000801040E05D2
:10695000054B02020E05054B04010E05054B050112
:106960000B04044B0801060303460000100002401C
:10697000080002400008024000000B00280002400E
:10698000080002400408024006010C0040000240DA
:10699000080002400808024010020D0058000240A2
:1069A000080002400C08024016030E00700002406E
:1069B0000C0002401008024000040F008800024052
:1069C0000C0002401408024006051000A00002401E
:1069D0000C0002401808024010061100B8000240E6
:1069E0000C0002401C08024016072F001004024051
:1069F0000804024020080240000838002804024031
:106A000008040240240802400609390040040240FC
:106A10000804024028080240100A3A0058040240C4
:106A2000080402402C080240160B3B007004024090
:106A30000C04024030080240000C3C008804024074
:106A40000C04024034080240060D4400A004024039
:106A50000C04024038080240100E4500B804024001
:106A60000C0402403C080240160F4600009600004D
:106A70000000000000000000000000000000000016
:106A80000000000000000000615000084D500008A8
:106A90008950000875500008815000086D500008AA
:106AA0005950000845500008955000086330000018
:106AB000AC6A0008186E0020287000200001002039
:106AC00000FF010002000000000000300000040090
:106AD000080000000000002400000800040000007E
:106AE0000004000000FC0000020000000000043070
:106AF00000800000080000000000003800000100D5
:106B0000010000006D61696E0069646C6500000041
:106B10000000002800000000AAAAAAAA0000002481
:106B2000FFFF0000000000000000000000A0550A68
:106B300000000000AAAA9AAA00500000FFF200007C
:106B40000000007700009900000000000000000035
:106B5000AAAAAAAA00000000FFFF0000000000008F
:106B6000000000005A000000000000009AAAAAAA33
:106B700000000000F3FF000099000000000000008A
:106B80000A00000000000000AAAAAAAA050000004E
:106B9000FFFF00008800000000000000000000006F
:106BA00000000000AAAAAAAA00000000FFFF00003F
:106BB00000000000000000000000000000000000D5
:106BC000AAAAAAAA00000000FFFF0000000000001F
:106BD000000000000000000000000000AAAAAAAA0D
:106BE00000000000FFFF00000000000000000000A7
:106BF0000000000000000000AAAAAAAA00000000ED
:106C0000FFFF000000000000000000000000000086
:106C100000000000AAAAAAAA00000000FFFF0000CE
:106C20000000000000000000000000000000000064
:106C3000AAAAAAAA00000000FFFF000000000000AE
:106C4000000000000000000013040000000000002D
:106C50000000180000000000FE2A0100D20400001D
:106C6000FF000000E86400205465002000000000E0
:106C7000686800088304000073680008500400007E
:046C8000816800081F
:00000001FF
